:1000000000000120B5020000DD020000DF02000058
:10001000E1020000E3020000E50200000000000031
:10002000000000000000000000000000E7020000E7
:10003000E902000000000000EB020000ED020000F9
:100040004D3A0000EF020000D1400000C94300001B
:10005000EF020000EF020000B13A0000EF020000E2
:10006000EF020000EF020000EF020000EF020000CC
:10007000EF020000EF020000EF020000EF020000BC
:10008000EF02000015160000EF020000EF02000072
:10009000B5160000EF020000EF020000EF020000C2
:1000A000EF020000EF020000EF020000EF0200008C
:1000B000EF020000EF02000000000000000000005E
:1000C000EF020000EF020000EF020000EF0200006C
:1000D000EF020000EF020000EF020000000000004D
:1000E0000000000000000000000000000000000010
:1000F0000000000000000000000000000000000000
:1001000000000000000000000000000000000000EF
:1001100000000000000000000000000000000000DF
:1001200000000000000000000000000000000000CF
:1001300000000000000000000000000000000000BF
:1001400000000000000000000000000000000000AF
:10015000000000000000000000000000000000009F
:10016000000000000000000000000000000000008F
:10017000000000000000000000000000000000007F
:10018000000000000000000000000000000000006F
:10019000000000000000000000000000000000005F
:1001A000000000000000000000000000000000004F
:1001B000000000000000000000000000000000003F
:1001C000000000000000000000000000000000002F
:1001D000000000000000000000000000000000001F
:1001E000000000000000000000000000000000000F
:1001F00000000000000000000000000000000000FF
:1002000010B5054C237833B9044B13B10448AFF350
:1002100000800123237010BD740200200000000044
:10022000006C000008B5034B1BB103490348AFF352
:10023000008008BD0000000078020020006C000073
:10024000154B002B08BF134B9D46A3F5803A0021A8
:100250008B460F461348144A121A05F08EFA0F4BBC
:10026000002B00D098470E4B002B00D09847002061
:10027000002104000D000D48002802D00C48AFF307
:10028000008005F02BFA2000290005F01BF805F08E
:1002900011FA00BF0000080000000120000000006B
:1002A0000000000074020020C809002000000000C7
:1002B000000000000649074A074B9B1A03DD043B78
:1002C000C858D050FBDC05F015F8FFF7B9FF000067
:1002D000C86C00000000002074020020FEE7FEE76A
:1002E000FEE7FEE7FEE7FEE7FEE7FEE7FEE7FEE7E6
:1002F000F0B595B0002415460F4608461E4603F09B
:10030000B9F9384623460895082205A91A9D099689
:100310000D950A948DF82C400C9403F025FA9DF865
:1003200014308DF81140DDE9061003F00302012AB4
:10033000CDE9020127D0022A04D0384603F09EF905
:1003400015B0F0BDBDF81650C3F3C2038DF81030E0
:10035000AD090826082D2C4628BF0824334622461E
:100360000EA9384603F000FA2D1B214608AB02AA5D
:100370000EA8264401F048F8002DEBD1384603F0D2
:100380007DF915B0F0BDBDF81460059DC6F3831668
:10039000C3F3C204B2000EA9384608238DF81040FA
:1003A000C5F3952503F0E0F908AB324628460EA9BF
:1003B000009302AB00F082FF384603F05FF915B0FE
:1003C000F0BD00BF704700BF00B583B0044B009381
:1003D000044A4023FFF78CFF03B05DF804FB00BF25
:1003E000E90300009402002038B50E480E4D037852
:1003F0000E4CEB5C0025D2B2257053B90C3004F0E2
:10040000D3FB58B90A4B1B7813B12378002BFCD0CF
:1004100038BD043004F0C8FE0028F3D001F0A0F885
:10042000F0E700BF00000020C4090020D402002033
:100430009002002070B51348134A0378D35C88B04B
:10044000DBB90C3004F020FB104D0FCD6C460FC40F
:1004500095E80F0008AD062645F8206D84E80F00EA
:1004600029460022074803F0B1FA08B101F078F8F4
:10047000074B00221A7008B070BD043004F000FE73
:10048000E2E700BF00000020C40900200858000077
:1004900090020020064B8B6004284FF00003CB60D5
:1004A0004B609CBF034B53F820300B60704700BF7C
:1004B000785A00009C5A0000C368DB6800225A7119
:1004C000704700BFC368DB6801225A71704700BFE4
:1004D00030B40E4B0E4D0F4CED1A00222D09C1E920
:1004E0000242C1E900220BD003EB0515DC68247938
:1004F000FF2C02D0904205D001321033AB42F5D12F
:1005000030BC70479B680B6030BC7047946C000037
:10051000A46C0000B05A00000129034604D0816891
:10052000D1F83C11890704D500221846114602F083
:10053000C9BA00B5D2E90031054A83B0CDE900213E
:10054000044A022101F044FF03B05DF804FB00BF40
:1005500004590000F85800008368D3F83C319B0729
:1005600033D42DE9F0471B4C1B4E361B360982B0A5
:1005700028D00746DFF868A0DFF86890DFF86880C9
:1005800004EB06160CE06D79CDF804C0002D0CBF0D
:1005900055464D460095103401F01AFFA64211D081
:1005A000D4E902E595F804C0BCF1FF0F734642465A
:1005B0004FF008013846E6D1084A103401F008FF30
:1005C000A642EDD102B0BDE8F0870022114602F04C
:1005D00079BA00BF946C0000A46C00003059000090
:1005E000245900001C590000505900008368D3F8BA
:1005F0003C319B0703D4044A022101F0E9BE0022EA
:10060000114602F05FBA00BF745900008368D3F846
:100610003C319B0703D4044A022101F0D9BE0022D9
:10062000114602F04FBA00BF74590000F0B5344CC7
:1006300085B004F5836001F06BFA04F2144001F018
:1006400067FAD4E9013703EA0702D01C04EB800102
:1006500014F8200010F0040042D003F1020C0E78D0
:1006600006F00306012E654635D0022E02F1030680
:1006700021D004EB86010028F1D104EB8202013382
:10068000D26801923B4004EB830302F00302012A8B
:10069000DE682ED0022A25D1BDF806309B0903332F
:1006A000360C05EB9305174801F03EFA00B1656082
:1006B000304605B0F0BD4B880CEB931307EA0302FC
:1006C000D11C03F1020C14F82100654604EB8101F2
:1006D00000F00400CFE70B88C3F383136344EDE716
:1006E0009D1CCAE708494FF4BF7001F0E1F90026EC
:1006F000D9E7BDF80430C3F38313360C1D44D2E7A9
:10070000A8030020BC070020885900002DE9F04113
:100710000F4C104D52F8046C2D1B2D0907460FD0BD
:1007200004EB051502E01034AC4209D0A168304654
:1007300005F02BF80028F6D1E3685871BDE8F08188
:1007400033463846044A0221BDE8F04101F040BE7C
:10075000946C0000A46C0000E05800002DE9F0410A
:10076000104C114D52F8046C2D1B2D09074610D06A
:1007700004EB051502E01034AC420AD0A168304603
:1007800005F003F80028F6D1E36801225A71BDE8AC
:10079000F08133463846054A0221BDE8F04101F0B8
:1007A00017BE00BF946C0000A46C0000E05800006D
:1007B00070B4104A104E114C921B0023D208C1E9AC
:1007C00002434B600CD00E4D2C88A04204D10CE0AB
:1007D00035F82340A04206D001339A42F8D10022D6
:1007E0000A6070BC704706EBC30632680A6070BCD2
:1007F000704700BF946C00003C6C0000785A000009
:100800001C0200202DE9F04FCB683E4EDFF820910E
:100810005B79A6EB090685B08B46F6088046002B6F
:100820006BD0394A394B0821404601F0D1FD384A96
:100830000821404601F0CCFD76B3364DDFF8F4A038
:10084000B70000240023EA5AA2423AD004339F4260
:10085000F9D15146002335F82320A24241D001337B
:100860009E42F8D100208446D646002335F8232046
:10087000A24223D001339E42F8D1002384450ED8F2
:10088000254A0292CDE9001E0134244A082140463F
:1008900001F09EFDA642D5D105B0BDE8F08F204AFB
:1008A0000292CDE9001E01341C4A0821404601F0A5
:1008B0008FFDB442C6D105B0BDE8F08F59F8333092
:1008C000DCE7DBF80C2017491279595802EB420299
:1008D000072393400B40D340DBB2134A52F8231056
:1008E000B8E709EBC30393F806C00F4B6046032833
:1008F00028BF032053F820E0B7E70C4A022101F09B
:1009000067FD8EE7946C0000F4590000E859000080
:10091000145A00001C02002070590000545A0000B4
:100920006C5A000048020020885A0000D459000088
:100930003C6C0000CC59000013460A46C168FFF722
:1009400061BF00BF2DE9F047124C134D52F8046C03
:100950002D1B2D09804615D01746894604EB051539
:1009600002E01034A5420DD0A168304604F00DFF1E
:100970000028F6D13B464A4621464046BDE8F047AE
:10098000FFF740BF33464046044A0221BDE8F04726
:1009900001F01EBD946C0000A46C0000E058000043
:1009A0002DE9F04F8E4B8F4C52F8049CA3EB0408BA
:1009B0005FEA181885B0064611D017460D4604EBBD
:1009C000081802E01034A04509D0A168484604F098
:1009D000DCFE0028F6D15DB905B0BDE8F08F824A93
:1009E0004B463046022105B0BDE8F04F01F0F0BCA7
:1009F000E3687E49386893F80490072204F0D7FE34
:100A0000002866D1012D00F0DE80DFF80C8204465C
:100A10000A2258F8041B786804F0C9FE58B1013462
:100A2000052CF5D17B68724A3046022105B0BDE83D
:100A3000F04F01F0CDBCE3B2022D019340F0BF8036
:100A40006C4C6D4BA3EB04085FEAD8082746C3D073
:100A500009EB490307229A400292019ADFF8A4A108
:100A60000194DFF8A4914FEA880802FA03FB0025FD
:100A7000144609E0019B53F8153001F0A9FC043538
:100A8000A84507F10807A7D0BB79A3424A464FF013
:100A900002013046EED355F80A20029982EA0B0390
:100AA0000B405340C3F3C202C3F382118A4238BFE2
:100AB0000A4603F007018A4238BF0A464F4945F803
:100AC0000A30C3F342206918824238BF02464A8086
:100AD000D5E708224A49386804F069FE00287AD12F
:100AE000012D0190ACD0012303F18043013B09EBC0
:100AF0004909A7F1040A07EB830707233D4C3E4A47
:100B000003FA09F30293019BA2EB04084FEAD80809
:100B100003FA09F3B3460AEB850A46460393A04657
:100B200057F8044F002E43D0C146002504E001359C
:100B3000AE4209F108093AD02022214658F8350082
:100B400004F035FE0028F2D1AE4230D099F80620EC
:100B5000019B9A4223D32B4C039B54F825200298E7
:100B60002649534003405340C3F3C202C3F38210EB
:100B7000824238BF024603F00700824238BF024675
:100B8000C3F3422001EB8501824238BF024644F89C
:100B900025304A80BA45C3D105B0BDE8F08FD9F8F9
:100BA0000030194A0221584601F012FCF2E73C6875
:100BB000164A23460221584601F00AFCEAE77FF66E
:100BC0000BAF022390E7124A3046022105B0BDE880
:100BD000F04F01F0FDBB3B680E4A304625E700BFF1
:100BE000A46C0000946C0000E0580000485800001D
:100BF000C05800003C6C0000946C00001C020020F7
:100C0000685800004802002088580000AC580000D6
:100C10005058000070580000885A000001B9704711
:100C20002DE9F04FC368DB6885B0894617468346D7
:100C30007A4910681D79072204F0B9FD00286ED1A9
:100C4000B9F1010F00F0DE80754E04460A2256F815
:100C5000041B786804F0ABFD58B10134052CF5D1C4
:100C60007B68704A5846022105B0BDE8F04F01F09C
:100C7000AFBBE3B2B9F1020F019340F0C0806A4C00
:100C80006A4F3F1BFF08264646D0019B029405EBA6
:100C900045051A46AA404FF0070A0AFA05FADFF896
:100CA0009891DFF898810192BF0000251C4609E069
:100CB000029B53F81530043501F08AFBAF4206F170
:100CC000080629D0B379A34242464FF002015846A4
:100CD000EED355F80920019B534003EA0A03534021
:100CE000C3F3C202C3F382118A4238BF0A4603F03B
:100CF00007018A4238BF0A464D4945F80930C3F317
:100D000042206918824205F1040538BF0246AF420D
:100D10004A8006F10806D5D105B0BDE8F08F08225B
:100D20004449386804F043FD002873D1B9F1010F3C
:100D30000190A4D0012303F18043013B05EB45055D
:100D40003A1F07EB83070723AB40374C374E02931C
:100D5000019B361BAB4002EB8909F6080393A046C2
:100D600057F8044F002E43D0C246002504E0013559
:100D7000AE420AF1080A3AD02022214658F835003E
:100D800004F015FD0028F2D1AE4230D09AF80620CA
:100D9000019B9A4223D3284C039B54F825200298A8
:100DA0002349534003405340C3F3C202C3F38210AC
:100DB000824238BF024603F00700824238BF024633
:100DC000C3F3422001EB8501824238BF024644F85A
:100DD00025304A80B945C3D105B0BDE8F08FDAF8B7
:100DE0000030164A0221584601F0F2FAF2E73C6858
:100DF000134A23460221584601F0EAFAEAE78BD962
:100E0000022398E70F4A5846022105B0BDE8F04F8B
:100E100001F0DEBA3B680C4A24E700BF48580000E6
:100E2000885A0000C05800003C6C0000946C000020
:100E30001C0200206858000048020020885800006A
:100E4000AC580000505800007058000021B9124BF7
:100E500003EBC00000687047104A0F49521AD208CD
:100E600015D030B40E4D2B88834212D0002303E0FE
:100E700035F82340844205D001339A42F8D100204E
:100E800030BC704701EBC300006830BC70471046AF
:100E900070470846F8E700BF3C6C0000946C000007
:100EA0001C020020094B013903EBC00003290BD8B9
:100EB000DFE801F00208060402207047407970471D
:100EC0000079704704207047002070473C6C000098
:100ED0002DE9F047DFF8FC90074600208846D9F856
:100EE000084000F0B1FDD9E90132D9F8006013449F
:100EF00001339B1B012B62D809F21C4501212846B6
:100F000000F0EEFDFFF792FB0146284600F0E8FDF9
:100F1000D9E90132D9F80010134401335B1A012BCF
:100F2000ECD90A40033205230231002049F822306F
:100F3000C9F8001000F0A2FD0021224800F0C6FD13
:100F400080F3100A204B214A3D0C9B1AB5EBD30FBE
:100F50002FD2731C234009EB83033440033445EA4A
:100F60000A45DD6019F8243067F3C50309F8243019
:100F700039F824306FF3891329F8243059F82420E4
:100F800068F39F221346012161F301036FF382038B
:100F900049F8242009F8243099F820341BB906E0D8
:100FA00000F01AF818B1D9E900329A42F8D1BDE838
:100FB000F087074940F2A31000F07AFDC9E73146F7
:100FC000AFE700BFC4070020946C00003C6C000039
:100FD00088590000A80300202DE9F04F9E4C002303
:100FE00085B0C4F81834BFF34F8FD4E9015605EA31
:100FF0000602D31C04EB830114F82330580719D5DB
:1010000027680B7803F00303012B3DD0022B03D19B
:101010004B88023505EB931506EA0502D4F818044F
:10102000D31C04EB830128B9AF423ED914F8233016
:101030005B07E6D404EB82026B1CD268019233405A
:1010400004EB830302F00302DB680293022A05F13A
:10105000020800F0A380012A2BD0D4F810543DB12F
:101060002B6828469B689847EB681D68002DF7D1D0
:101070007A4B5B88012B0DD8D4E90030C01A18BF19
:10108000012005B0BDE8F08F0B880235C3F3831350
:101090001D44C1E7724B73487349C01AC00800046D
:1010A00040F00200FFF714FFE6E7676005B0BDE817
:1010B000F08FBDF804706D48C7F38313062B28BF6B
:1010C0000623991C63F389178900ADF8047002F0B8
:1010D0008FFAC7F3C20781460028BED002F0CAFAD1
:1010E0000023082201A9484602F0EAFABDF80430BC
:1010F00013F4707F00F0AE806FF0010BABEB050BCB
:10110000082506EA080103312B46042204EB81017D
:10111000484602F0D5FABDF8043008F1010A0BEB9D
:101120000A02C3F383139342D04605F10405E8D8BD
:10113000D4F81834002B77D1D4F81054FDB1DFF86F
:1011400034810726EB685A79B2B11A79BDF80800E4
:1011500002EB420158F8200006FA01F2052F02EADC
:10116000000208BF0327CA40BA4205D32B6849468C
:101170001B6828469847EB681D68002DE2D1484659
:1011800002F07CFA002000F05FFCD4F818340BB9B0
:10119000C4F804A0002000F071FC6DE7BDF8063033
:1011A00032489DF804704FEA931A5546502D28BFD7
:1011B000502565F38F1305F10801ADF8063002F0F4
:1011C00017FAC7F3C207814600283FF446AF26EA64
:1011D000080B0BF1010B02F04DFA4FEA8B0B0023C9
:1011E000082201A9484602F06BFA5D4527D9EBB207
:1011F000BBF1000F1CD006EA0801A3EB0B0303317F
:1012000004EB8101DDB25A460823484602F058FA41
:101210002A460BF108031649484602F051FA0AF132
:10122000030A08EB9A0A83E7484602F027FA23E705
:101230002A4608230E49484602F042FAEFE706EA3A
:101240000801033104EB81012A460823484602F0D5
:1012500037FAE4E7C2466BE7A80300203402002017
:101260003C6C00006C6C0000F85B0000A46C00009B
:10127000B403002048020020044BD3E900239A4223
:1012800001D0FFF7A9BE0020704700BFA8030020CF
:1012900038B5094BD3F81044012583F820544CB1DC
:1012A000E3685D71236820465B689847E3681C68C3
:1012B000002CF5D138BD00BFA80300202DE9F04770
:1012C00084B01D460C9C002394F80C802373EB889B
:1012D00081460E461746002B40D1297A05290ED0AB
:1012E0006B7AA88873BB404B53F821A00021FFF70D
:1012F000ADFD524603463D49204601F0B3FD062FA1
:1013000009D8DFE807F0046A4249525D33004946D4
:10131000204601F0A7FD2B7A052B05D06B7A5BB92F
:101320003349204601F09EFD204601F087FD84F8F8
:101330000C8004B0BDE8F0872E4A2F49204601F00A
:1013400091FDEDE7FFF7AEFD2C4B2B4953F8202024
:10135000204601F087FD297AA888C4E7254A009233
:101360002749284A204601F07DFDB6E7D6E904105A
:10137000D6E900230390D6E902070291CDE90007E0
:101380004946204601F06EFDC5E74946D6E90023EF
:10139000204601F067FDBEE7B168D6E9002320468C
:1013A0000091494601F05EFDB5E7D6E90201D6E9B4
:1013B0000023019100904946204601F053FDAAE721
:1013C000D6E90371B068D6E900230291CDE90007A0
:1013D0004946204601F046FD9DE7326849462046D1
:1013E00001F040FD97E700BFFC5E0000F05E0000EA
:1013F0004C590000E85E000094640000905E00001C
:10140000D05E0000C85E0000082900D970472DE9B1
:10141000F04F1D46904600232A7B2B7385B0B8F809
:101420000630039207460E46002B77D198F8081035
:10143000052911D098F80930B8F80400002B5FD1C5
:101440003A4B53F821400021FFF700FD22460346A6
:101450003749284601F006FDDFF8F4B0DFF8F490D4
:10146000002405E03A5D013401F0FCFC082C09D0B1
:10147000A64249462846F5D85946013401F0F2FC07
:10148000082CF5D12B49DFF8D090DFF8D0B02846F2
:1014900001F0E8FC002411E017F804A004F042F980
:1014A00050445946437813F0970F14BF52462E22EA
:1014B0002846013401F0D6FC082C08D0A642494643
:1014C0002846E9D8013401F0CDFC082CF6D198F873
:1014D0000830052B02D098F809305BB91649284628
:1014E00001F0C0FC284601F0A9FC039B2B7305B05A
:1014F000BDE8F08F114A1249284601F0B3FCEDE730
:10150000FFF7D0FC0F4B0E4953F82020284601F07E
:10151000A9FC98F80810B8F8040091E7074A00926F
:1015200009490A4A284601F09DFC7FE7FC5E00005D
:10153000F05E0000C05E00004C590000E85E000054
:1015400094640000905E0000D05E0000C85E000061
:10155000BC5E0000B45E0000F85E0000C45E0000E7
:1015600000B585B000230390194601AA44F201009A
:10157000CDE9013300F004F805B05DF804FB00BFCD
:1015800070B572B6FFF784FEFFF776FE0028FBD138
:10159000184E7388F3B9184B1B68DB070DD5174C31
:1015A000174D00BE7388012B07D9601BC0080004CB
:1015B00040F002001349FFF78BFCBFF34F8F124935
:1015C000124BCA6802F4E0621343CB60BFF34F8F43
:1015D00000BFFDE7094C0A4D0D49601BC00800041F
:1015E00040F00100FFF774FC034B1B68DA07D9D504
:1015F000D7E700BF34020020F0ED00E06C6C000083
:101600003C6C0000545F000000ED00E00400FA05AF
:10161000485F0000F8B5204A204B0024C2F8404142
:10162000C2F84441C2F84841C2F84C41C2F80041F6
:10163000C2F804411B6833B31949D2F804550A684B
:10164000AD1A1A6825F07F45AA4227460DD8197CA5
:10165000DE69AD1A144419B11F74D3E9052090470F
:101660001EB133461A68AA42F1D90E490E4A0B78C8
:1016700012789A4208D00D490D4A41F823404FF4A0
:101680008013C2F80031F8BD531CDBB2022B08BF37
:1016900000230B70EFE700BF00100140EC080020B2
:1016A000E8080020E5080020E4080020DC0800200D
:1016B00000E100E02DE9F04F8C4A8D49137809785C
:1016C000DFF85082994285B0D8F800A000F07B8105
:1016D0000133DBB2022B08BF002386481370864A11
:1016E000076852F823107B1823F07F43002403601F
:1016F000534626462046A446ABB11A688A4200F2F9
:101700006581DC68C3F800C0891A1044DA6934B115
:101710003D1825F07F45C3E90154DE611E4613469E
:101720000124002BE9D1002C40F07C81012300939F
:10173000724B734FDFF8E09143F00103019355467C
:101740004FF0000B46B3D6E901C13446F669694B48
:101750006C481A68ACEB020323F07F43834248D8FD
:101760000B44236000220121C4E90122E2612174BB
:10177000002D5DD02A689A424DD2284603E00A68BF
:101780009A424FD20846C1699B1A0029F7D12360BB
:10179000E161C461002ED6D178783978884264D06E
:1017A0000B4603EB43034C1CBA7807EBC303E1B2CF
:1017B0008A421A79397004BF00213970022A9C6864
:1017C00044D0032A38D0012AE8D1227C002AE5D16E
:1017D000D3F80CC0C4F804C01969A1605869E0606E
:1017E00099F800009B69A3610028B0D0626094461C
:1017F000ADE7A2EB0C0222F07F428A4202D28B1AA2
:101800002360AFE700230122C4E90033A360E36152
:1018100022746DB12A68C8F80040D31A2B60E561C4
:1018200025468FE7D21A0A602360E161C461B1E7FF
:10183000C8F80040254685E7002DAFD000232B7463
:10184000ED69002DFBD1C8F80050A5E74DB1AC42C1
:101850002B4603D1E4E094422FD01346DA69002AE4
:10186000F9D10023237488429AD1BBF1000F01D132
:10187000554553D0002D56D1234E244A1F4C4FF4CA
:1018800080334FF400310127C2F880103C43C6F882
:1018900048334FF43C60C6F808337760A047154BD7
:1018A000B7604FF43C601D60A047194B1D700023CA
:1018B00089F8003005B0BDE8F08FA34200F09180B8
:1018C000E0692168D861002800F086802A46036814
:1018D0000B440360AA424FF00003397878782374F0
:1018E0001CBF15464FF0010BBDE700BFE408002008
:1018F000E5080020E8080020DC080020705F0000F8
:10190000CC070020FEFF7F000010014000E100E056
:10191000D9080020EC080020D8080020009B002BEC
:10192000C5D0002DA8D0434B434A1C68D2F80465AB
:10193000424FD5F800A03978331B23F07F43DD1CDC
:10194000B9B93F493F4B4FF48030C2F844034FF0E0
:101950000108C2F804034FF40030C1F8800143F0DD
:1019600001030860C2F800804FF43C60984787F894
:101970000080AA452CBF04EB0A0363192E4923F00B
:101980007F43C1F84035D1F80425921B9B1B22F000
:101990007F4223F07F4303329A4288D9294BD1F802
:1019A0000425C1F8402543F001034FF43C609847FB
:1019B000234B4FF40032C3F80021002389F8003094
:1019C00005B0BDE8F08F00260096B1E674BB521A50
:1019D0001A6001230093ABE60023397878782374EA
:1019E00041E71946EA69C8F8002092B9CDE9023109
:1019F000114BDFF840C001209860019B89F800007E
:101A0000CCF800204FF43C609847DDE90231D8F86B
:101A10000020C8690968D86100287FF458AF59E7E9
:101A20002946DFE7C8F800309A467FE6C8F800305C
:101A30009A46CCE7E808002000100140D9080020B1
:101A400000E100E0705F000008B5EFF30583C3F329
:101A500008032BB172B6074A13680133136008BD3F
:101A6000EFF31483DB07F5D50349432000F020F89A
:101A7000F0E700BFF0080020785F000008B5EFF342
:101A80000583C3F3080333B1074A1368013B1360AE
:101A900003B962B608BDEFF31483DB07F4D503493D
:101AA000512000F005F8EFE7F0080020785F000013
:101AB00000B583B06A46ADF80000019144F202001F
:101AC0000021FFF75DFD03B05DF804FB50E8002F37
:101AD0000B4640E8003C9CF0000FF7D110467047E1
:101AE00050E8003F03EB010240E8002C9CF0000F9F
:101AF000F6D11046704700BF50E8003FA3EB01024B
:101B000040E8002C9CF0000FF6D11046704700BF53
:101B1000012350E8002F42EA030C40E800C191F095
:101B2000000FF6D160467047002350E800CF0CEA62
:101B3000030240E8002191F0000FF6D160467047A3
:101B40002DE9F0438368D3F83C61C6F340068BB0BF
:101B5000002E47D101293ED8264C274D274B2D1B5F
:101B6000AD08A3FB0535002D32D0C5EBC505DFF868
:101B70009490074604EB85054FF064082368A1683C
:101B80001A7918686369099363680692081A02EB68
:101B90008202A1EB030CC0B2218B039002EB820204
:101BA00000910196920008FB00F0B2FBFCF2B0FB42
:101BB000FCF005920290CDF81CC0CDF810C0099B36
:101BC0001C344A460821384600F002FCA542D5D113
:101BD0000BB0BDE8F0830A4A02210BB0BDE8F04328
:101BE00000F0F6BB002211460BB0BDE8F04300F058
:101BF00069BF00BFA46C0000C06C0000254992249E
:101C00001C6000003060000038B50446E8B10020D8
:101C1000FFF71AFFD4E900311A688A421BD9511E16
:101C200019602168A3680868258B12F8012CE46804
:101C30001B1A0879DBB2984205FB024400D20B71F3
:101C40000020FFF71BFF204638BD04494FF4927077
:101C5000FFF72EFFDBE70024F2E700BFE05F0000A4
:101C600038B50C46054690B1C4B10020FFF7ECFE34
:101C70002A681368591C1160E9682A8B641AB4FB3E
:101C8000F2F41C700020BDE83840FFF7F7BE0649AB
:101C900040F24710FFF70CFF002CE6D102494FF449
:101CA000A470FFF705FFE0E7E05F00002DE9F047D3
:101CB000884682B01446054600283BD0002939D01A
:101CC0006B681B68002B3DD08CB3DFF88490002735
:101CD0004646686803682246D3F80CA0314601AB3B
:101CE000D047F8B9019BA34206D863B1E41A1F4458
:101CF0001DD008EB0706ECE74946F420FFF7D8FEB5
:101D0000019B002BF2D1AA681378032BE1D0D2F803
:101D10003C319B06FBD592F83C316FF3451382F8BA
:101D20003C31D6E74946F320FFF7C2FEDAE702B0BE
:101D3000BDE8F0870649E820FFF7BAFE6B681B682C
:101D4000002BC1D10249E920FFF7B2FEBCE700BF7A
:101D50001C6100002DE9F04305468068504F83B0B8
:101D600000268022314694308DF8036003F005FD93
:101D700028694C4901F076F8286901F05FF847F0CE
:101D800001074FF47A79DFF820816868002833D0A2
:101D9000036801221C690DF1030101ABA047019BFF
:101DA0004FF6C01063B9B847019B002BEDD109F184
:101DB000FF391FFA89F9B9F1000FE4D10D2018E0BD
:101DC0009DF80330AA681B2B06F1010002EB060107
:101DD00005D092F894401B2CD7D1522B13D0C6B209
:101DE000092E81F89430D0D9AB68002283F8942072
:101DF000042003B0BDE8F0834FF48C704146FFF738
:101E000057FE6868C4E7002681F89460AF6897F8C9
:101E100095305B2B3AD107F19504022302E0802B29
:101E200096B239D014F8010F0133A0F1300106EB5E
:101E30008602DBB23B2801EB420259B2EFD1002906
:101E40002ADB03F1930CBC44002002E090B21A0696
:101E500022D41CF8014F00EB80020133A4F13001C1
:101E600001EB4202DBB2002CF0D1FA2828BFFA20A5
:101E70003872AB68FA2E86BFFA229A729E72AB68ED
:101E8000002083F8940003B0BDE8F0830B2087F8AE
:101E9000946003B0BDE8F0830C2003B0BDE8F0838C
:101EA000A0610000706100001C6100000CB430B53E
:101EB00085B00446089D002D54D0002C59D0A1684F
:101EC000B1B16368A3B1236893B109AB0193D1F8B1
:101ED0003C315B0702D5CB7B082B10D1294620690A
:101EE00001AA01F077F805B0BDE8304002B07047B4
:101EF000364940F64B30FFF7DBFDA168E5E70222EB
:101F00000F31684603F02EFCA368DA7B082A36D12D
:101F100001AA2946206901F05DF89DF80030A26809
:101F2000002B4BD0D17B994235D19DF80130002B4D
:101F3000D9D0A268117C9942D5D045F61B3103F166
:101F40002F00ADF8081034256D218DF80B00ADF889
:101F50000C108DF80A50137420691D4902AA00F074
:101F600081FFC0E7194940F64930FFF7A1FD002C79
:101F7000A5D1164940F64A30FFF79AFD9FE7154A6A
:101F80000292154903910822DA73206910496A44C4
:101F900000F068FFBCE70F49029103F12F003325E1
:101FA0006D218DF80D00ADF80E108DF80C50D37327
:101FB0002069074902AA00F055FFB6E7D3732069EC
:101FC000064A034900F04EFFAFE700BF1C61000066
:101FD000946400001B5B313B33376D005861000097
:101FE000002900F0B5802DE9F04F884683B01646F1
:101FF00005464F1E002400E0013403F093FB17F860
:10200000013F184443781907F6D4F3B20193A2466E
:10201000404603F0C4FBAB6893F80DB0A0EB0A0098
:10202000ABEB060B58454AD90AF1FF3208EB020424
:10203000002700E0013703F075FB14F8013F184456
:10204000F119427812070AEB070902D50A2B07D0CB
:10205000BB46AB685B7B9942ECD30AEB0B095F464E
:10206000286900F0EBFE3A4608EB0A01284609F120
:10207000FF37FFF71BFE474401E009F1010903F0B8
:1020800051FB17F8013F184443781B07F5D4286922
:1020900070B1334A334900F0E5FE019B0BB9CA46E3
:1020A000B6E71A463049286900F0DCFECA46AFE7B9
:1020B0004FF4ED702D49FFF7FBFC2869E9E7544622
:1020C000C24478B118F804300A2B18D053460026C1
:1020D00003E013F8012F0A2A13D00136B04204EBB3
:1020E0000607F6D12869514600F0BCFE286940B3C6
:1020F0001B4A1C4903B0BDE8F04F00F0B3BE2746B1
:102100000026286900F09AFE284632465146FFF71D
:10211000CDFD28690137E0B1114A124900F0A2FE55
:10212000019B08EB070A002BDCD01A460E492869F0
:1021300000F098FE2869514600F094FE28690028B6
:10214000D6D14FF4ED700949FFF7B2FC2869CFE70B
:1021500070474FF4ED700549FFF7AAFC2869DBE7EB
:1021600054610000946400008C6100001C61000058
:102170002DE9F047044686B0002800F0C080A3682F
:10218000002B65D06368002B62D02368002B5FD0E2
:102190005E4803F004FB05465D4803F000FBA368BE
:1021A0005C495B685C4A1B6800912D1A0821204637
:1021B000FFF77CFEA3685B681868ADB2002800F0EA
:1021C000918003F0ECFA86B2524803F0E8FAA36873
:1021D0005B683044596882B22046FFF701FF4F4ADE
:1021E00008212046FFF762FE494803F0D8FA023082
:1021F0000544ADB2454B0093494A2B460821204681
:10220000FFF754FEEA1C92B246492046FFF7E8FE6B
:10221000A3685B689D68002D59D000231E462A786C
:10222000D5F8048002A918465F1CBAB1C0470298CD
:10223000D8B10DF1080903F0B2FAB04206D9D9F8C5
:102240000060304616B103F0AAFA86B23B46E6E7D4
:10225000354940F6CB30FFF72BFC99E71B0108EB23
:10226000030958F803000028E5D1012F2FD02F4A89
:10227000DFF8ACA020460821FFF718FE2A786B682B
:1022800006F1020900201FFA89F900F10108CAB11C
:1022900002A99847029BD3B102AF009308214B4695
:1022A00052462046FFF702FE796899B1721D20461A
:1022B00092B2FFF795FE40462A786B6800F101085C
:1022C000002AE5D100011F181B58002BE5D106B0EC
:1022D000BDE8F087206938B1154A164900F0C2FD03
:1022E0004046E9E706466FE70F494FF4ED70FFF708
:1022F000DFFB20690E4A0F4900F0B4FDF0E70A4900
:1023000040F6CA30FFF7D4FB39E700BFA8610000F0
:10231000B064000078610000E4630000A86300007E
:10232000B4630000BC6300001C610000D0630000C7
:10233000546100009464000038B50D46044630B383
:10234000A3689BB163688BB123687BB1022D14D065
:10235000206910B31A4A1B4900F084FD206918B3A4
:10236000194A1849BDE8384000F07CBD174940F6CD
:102370004E50FFF79DFB022DEAD1A368D3F83C3104
:102380009B07E5D52046BDE83840FFF7F1BE0F4971
:1023900040F64D50FFF78CFBD2E740F656500B4904
:1023A000FFF786FB2069D5E7084940F65750FFF74D
:1023B0007FFB2069044A0349BDE8384000F052BD64
:1023C0005C61000094640000606100001C6100001A
:1023D0000CB470B584B00446089D0E46002D56D04E
:1023E000002C5BD0A168B1B16368A3B1236893B13D
:1023F00009AB0193D1F83C315B0702D5CB7BB342EB
:1024000010D12946206901AA00F0E4FD04B0BDE81E
:10241000704002B070473E4940F64B30FFF748FB32
:10242000A168E5E70F310222684603F09BF9A36833
:10243000002E66D0DA7BB24236D101AA2946206945
:1024400000F0C8FD9DF80030A268002B52D0D17B6F
:1024500099423CD19DF80130002BD7D0A268117C65
:102460009942D3D045F61B3103F12F00ADF8081087
:1024700034256D218DF80B00ADF80C108DF80A5045
:1024800013742069234902AA00F0ECFCBEE720493E
:1024900040F64930FFF70CFB002CA3D11C4940F655
:1024A0004A30FFF705FB9DE71B4A0292332206F1F3
:1024B0002F018DF80C206D228DF80D10ADF80E2037
:1024C000DE732069134902AA00F0CCFCB5E712497B
:1024D000029103F12F0033256D218DF80D00ADF829
:1024E0000E108DF80C50D37320690A4902AA00F02F
:1024F000B9FCAFE7D3732069084A064900F0B2FC83
:10250000A8E7DE732069054A024900F0ABFC94E7B6
:102510001C610000946400001B5B313B58610000AB
:1025200038B50D46044608B3A3689BB163688BB108
:1025300023687BB1012D14D0022D04D1A368D3F8F8
:102540003C319B070DD420460B4A0221BDE83840A0
:10255000FFF73EBF094940F65D50FFF7A9FA012D8C
:10256000EAD12046BDE83840FFF702BE034940F6F5
:102570005C50FFF79DFAD7E73C6400001C61000047
:10258000F0B50E4683B01746044600286CD0A56807
:10259000BDB16368ABB123689BB1012E19D0D5F8EA
:1025A0003C319B0754D4022E64D8D7E900313C4A11
:1025B0000191009220463B4A0221FFF709FF03B038
:1025C000F0BD394940F62C60FFF772FA012EA5687C
:1025D000E5D115F10D0F05F10C063FD0002E53D0BB
:1025E0002046FFF7B7FB28BBA368304920691F7A54
:1025F0009E7AFA2200F036FC20692D49FA2200F07A
:1026000031FC2046FFF7A6FBA0B9A3681A7A6A73CB
:10261000A368D21B9B7A2B7312F0FF023AD19B1B4B
:1026200013F0FF02CBD02069224903B0BDE8F0408F
:1026300000F018BCA368204A50215973A3681821E0
:1026400019732046042103B0BDE8F040FFF7C0BE77
:10265000204603B0BDE8F040FFF78ABD124940F2C2
:102660003D30FFF725FAB9E70F4940F62B60FFF739
:102670001FFA8CE76B68114A1B682046022103B0E1
:10268000BDE8F040FFF7A4BE074940F23E30FFF737
:102690000FFAA5E70A49206900F0E4FB2B7BBEE7AF
:1026A00004590000F85800001C6100008C61000013
:1026B0007C61000094610000506300008C630000A6
:1026C000846100008368D3F83C2192070ED401296D
:1026D00006D193F83C2142F0080283F83C21704770
:1026E0005B68034A1B680221FFF772BEFFF740BD1B
:1026F0008C6300008268D2F83C31C3F3400373B9A5
:10270000012906D192F83C1163F3C30182F83C1110
:1027100070475368034A1B680221FFF759BEFFF751
:1027200027BD00BF8C6300008268D2F83C31C3F340
:1027300040038BB9012909D110B4C2F82C31C36808
:102740005DF8044B5B68186801F0FAB85368034AF7
:102750001B680221FFF73CBEFFF70ABD8C63000037
:1027600030B58268D2F83C41A30785B026D4012950
:102770001BD1C3685B681D680446284601F0D0F889
:10278000A368A968D3F82C310291C0B2642202FB7D
:1027900000F2B2FBF1F2D2B2CDE9002008212046CE
:1027A000094AFFF783FB05B030BD5368074A1B6831
:1027B000022105B0BDE83040FFF70ABE05B0BDE814
:1027C0003040FFF7D5BC00BFEC6200008C63000016
:1027D00010B58268D2F83C41A30717D401290DD166
:1027E00004460069B0B10F4A0F4900F03BFBA368F3
:1027F00050225A73A36818221A7310BD53680B4AEB
:102800001B680221BDE81040FFF7E2BDBDE81040A3
:10281000FFF7AEBC40F624600549FFF749F920698F
:10282000E1E700BF68610000946400008C63000071
:102830001C6100008268D2F83C31C3F3400373B9D5
:10284000012906D192F83C1163F3820182F83C1110
:1028500070475368034A1B680221FFF7B9BDFFF7B1
:1028600087BC00BF8C6300008368D3F83C219207CB
:102870000ED4012906D193F83C2142F0040283F8DA
:102880003C2170475B68034A1B680221FFF7A0BD2B
:10289000FFF76EBC8C63000030B58368D3F83C4111
:1028A000A40783B01AD402290FD81CD0D3F83C4116
:1028B0001249134B134A14F0080F18BF0B46082196
:1028C00003B0BDE83040FFF7F1BA5B680E4A1B6801
:1028D000022103B0BDE83040FFF77ABD03B0BDE888
:1028E0003040FFF745BCD2E90034084ACDE9002466
:1028F000074AFFF76DFD03B030BD00BF286300003D
:102900002C630000306300008C6300000459000059
:10291000F8580000F0B50E4687B0054600284ED0A6
:10292000AB6893B36A6882B32A6872B3D3F83C4148
:10293000C4F34004002C34D1012E37D1D3F83461D4
:10294000F6B1224F30460023092203A900F00CFF04
:102950009DF81420A968304601329431092300F013
:1029600003FFAB68049E943300933A462346082144
:1029700028460134FFF79AFA0EB1082CE2D1AB6871
:10298000002283F8942007B0F0BD114940F6C450EE
:10299000FFF78EF8AB68D3F83C41C4F34004002C39
:1029A000CAD02846FFF7E4FB07B0F0BD5B68094AD0
:1029B0001B6828460221FFF70BFD07B0F0BD044954
:1029C00040F6C350FFF774F8AAE700BF4463000065
:1029D0001C6100008C63000070B50D4682B0164685
:1029E0000446002830D0A368F3B16368E3B12368DC
:1029F000D3B1012D12D0A368D3F83C2192070DD496
:102A0000022D17D1D6E90031124A019100922946D0
:102A10002046114AFFF7DCFC02B070BD204602B030
:102A2000BDE87040FFF7A4BB0C4940F67E50FFF7AD
:102A30003FF8DEE75B680A4A1B682046022102B0C5
:102A4000BDE87040FFF7C4BC044940F67D50FFF775
:102A50002FF8C8E704590000F85800001C61000076
:102A60008C63000010B5012982B004460BD0022906
:102A70000B460ED08268D2F83C11890703D4022B92
:102A800011D802B010BD204602B0BDE81040FFF7DB
:102A90006FBBD2E90034084ACDE90024074AFFF7AA
:102AA00097FC02B010BD5368054A1B68022102B0B2
:102AB000BDE81040FFF78CBC04590000F858000036
:102AC0008C6300002DE9F04F0C4687B09146054617
:102AD000002800F09F81AB68002B61D06B68002B51
:102AE0005ED02B68002B5BD0AC4802F058FE064647
:102AF000AB4802F054FEAB68AA495B68AA4A1B685F
:102B00000091361A08212846FFF7D0F9AB685B68B8
:102B10001868B6B2002800F0C38002F040FE87B209
:102B2000A04802F03CFEAB685B68384482B259684A
:102B30002846FFF755FA9D4A08212846FFF7B6F9BF
:102B4000B9F1000F32D0002C00F0448109EB4909A3
:102B500004EB890927461BE0184602F020FE804658
:102B6000386808B102F01BFE4044B0420CD97868C6
:102B7000002800F0978002F012FE86B2386818B183
:102B800002F00DFE0644B6B20C37B94500F08C8059
:102B90007B68002BE0D138680028F5D09846E1E743
:102BA000834940F6CB30FEF783FF9DE77C4802F077
:102BB000F6FD02300644B6B2784B00937D4A3346A8
:102BC000082128460336FFF771F9B2B27A49284640
:102BD000FFF706FAAB685B689C68002C53D00023B3
:102BE0001E462278D4F8048002A918465F1C8AB1D8
:102BF000C0470298A8B10DF1080902F0D0FD864245
:102C000006D2D9F80060304616B102F0C8FD86B28F
:102C10003B46E6E71B0108EB030958F803000028D0
:102C2000EBD1012F2FD0654ADFF888A12846082173
:102C3000FFF73CF92278636806F1020900201FFAC9
:102C400089F900F10108CAB102A99847029BD3B1E2
:102C500002AF009308214B4652462846FFF726F95B
:102C6000796899B1721D284692B2FFF7B9F94046CA
:102C70002278636800F10108002AE5D100011F18DD
:102C80001B58002BE5D107B0BDE8F08F286900285C
:102C900000F0B5804A4A4B4900F0E4F84046E7E7C7
:102CA00007463DE7064669E73D4802F078FD00F13A
:102CB0000208B0441FFA88F8384B009308F1030962
:102CC00043463C4A082128461FFA89F908F1020ABE
:102CD000FFF7ECF85FFA8AFA4A4637492846FFF7C9
:102CE0007FF9AAF1020A2EE02D492846CDE900120B
:102CF000354A0821FFF7DAF8606800283FD002F073
:102D00004EFDC6B22068002837D002F048FD5FFAB9
:102D100080FB234802F043FDAAEB0606A6EB0B025C
:102D2000121A12F0FF022CD13A222849286900F029
:102D300099F8A168B1B14A462846FFF751F90C3419
:102D4000BC423FF447AFD4E9002393B1002ACBD172
:102D5000009308214346174A2846FFF7A7F8A168C1
:102D60000029E8D1286988B1154A164900F07AF897
:102D7000E5E7002ADDD00092EBE78346C9E7064687
:102D8000C0E71349286900F06DF8CDE74FF4ED7006
:102D90000749FEF78DFE2869E6E700BFA86100003D
:102DA000B064000078610000E4630000A8630000E4
:102DB0001C610000B4630000BC630000D06300002D
:102DC0005461000094640000E0630000C45E0000F1
:102DD0008C610000124802F0E2FC02300644B6B2F8
:102DE000104B0093284633460F4A0821FFF75EF840
:102DF000F21C92B20D492846FFF7F2F8EAE60C49B8
:102E00004FF4ED70FEF754FE28690A4A0A4900F0B3
:102E100029F843E7064940F6CA30FEF749FE5AE66C
:102E2000B0640000A8610000B4630000BC6300004F
:102E30001C610000546100009464000010B5044659
:102E400040B1A2682AB163692168206998470023CC
:102E5000A36010BD02493120FEF72AFEF1E700BF52
:102E60006C6700000EB430B582B00446059DE8B131
:102E7000636913B32368A3B163686BB13DB102AA60
:102E800006AB42F8043D2946204600F0A3F802B004
:102E9000BDE8304003B070470A494520FEF708FE00
:102EA000ECE708494420FEF703FEE5E70549422028
:102EB000FEF7FEFD6369002BDCD102494320FEF7DB
:102EC000F7FDD7E76C6700002DE9F84F884690457D
:102ED000174605461E46DDE90AB175D343464FF055
:102EE0000109B3FBF7F39F4209F10109F9D9B14593
:102EF00038BFB14611F0010AAA6802D1BBF1000F38
:102F000043D1012402E0013E07FB04F4012EFAD86C
:102F1000B8FBF4F18F42F7D92D4E05E0B4FBF7F47E
:102F2000A4B1B8FBF4F1AA68705C531CAB602B68C9
:102F30009854D5E901329A4204FB1188EED3284611
:102F4000FFF77CFFB4FBF7F4002CEAD1BAF1000FD5
:102F500015D0BBF1000F12D0CB4510D92024AB689F
:102F60002A68591CA960D454D5E901329A420BF160
:102F7000FF3B06D2BBF1000F01D0CB45EFD1BDE83E
:102F8000F88F2846FFF75AFFF4E78B0717D4202461
:102F9000CB45B6D92B68511CA9609C54D5E90132A8
:102FA0009A420BF1FF3B05D2BBF1000FA9D0CB45F4
:102FB000F0D1A6E72846FFF741FFAA68F4E7002E04
:102FC0000CBF30242024E3E74FF001098FE700BF56
:102FD000A06700002DE9F04F0D4685B092460446EB
:102FE000002800F004826369002B00F00982236846
:102FF000002B00F00E826368002B00F03381E5B1F6
:103000002B78DFF85CB501E02B7893B1013583B103
:10301000252B15D0A2682168501CA0608B54D4E9E0
:1030200001329A42F0D32046FFF708FF2B78002B9D
:10303000ECD1237B002B40F01B8105B0BDE8F08F65
:103040002946002711F8012B2D2A00F0E280302AB2
:1030500000F0E3802B2A00F0D3802A2A00F0E180E0
:10306000A2F13006F3B2092B03D9D8E1A3F130065F
:103070000146084606EB860310F8012BA2F1300545
:10308000092D02EB4303F1D92E2A00F0D68000234C
:10309000013101E011F8012B02F0FB0068280D4618
:1030A000F8D0253A532AAFD801A151F822F000BF39
:1030B0007D320000093000000930000009300000B6
:1030C000093000000930000009300000093000001C
:1030D000093000000930000009300000093000000C
:1030E00009300000093000000930000009300000FC
:1030F00009300000093000000930000009300000EC
:1031000009300000093000000930000009300000DB
:1031100009300000093000000930000009300000CB
:1031200009300000093000000930000009300000BB
:1031300009300000093000000930000009300000AB
:10314000093000000930000009300000093000009B
:10315000093000000930000009300000093000008B
:10316000093000000930000009300000093000007B
:1031700009300000093000000930000097320000DB
:10318000093000000930000009300000093000005B
:10319000093000000930000009300000093000004B
:1031A0000930000009300000B1320000D3320000C5
:1031B000093000000930000009300000093000002B
:1031C000D33200000930000009300000093000004F
:1031D00009300000093000000930000025330000EC
:1031E0000930000009300000993300000930000068
:1031F000D53300000930000009300000973200008C
:1032000047F004070D46294611F8012B2D2A7FF4BB
:103210001EAF47F001070D46F5E747F002070D46E0
:10322000F1E7DAF800301A1DCAF800206A781E6843
:103230002E2A05F102007FF42AAF4A78A2F130036A
:10324000092B00F27081002303EB830302EB43039D
:1032500010F8012FA2F130010929A3F13003F3D9AD
:10326000014615E7BC494FF4A170FEF721FCC6E604
:10327000204605B0BDE8F04FFFF7E0BDA368226827
:10328000591CA1604FF02501D154D4E901329A4272
:10329000FFF4BAAEC7E6DAF80020111DCAF8001034
:1032A00011682046CDE900671022FFF70DFEABE65E
:1032B000DAF80020131DCAF80030A36821681278DC
:1032C000581CA060CA54D4E901329A42FFF49CAE63
:1032D000A9E6DAF80020111DCAF80010D2F8008023
:1032E00088EAE872A2EBE872092A4FF0010107DDD3
:1032F0009A48A0FB0202D208092A01F10101F7DC79
:10330000994238BF1946894607F00202002E40F064
:103310008A802AB1002B00F06781FA0700F1A680AD
:103320000026A3E0DAF80020131DCAF80030A368D5
:1033300021681768581C3022A060CA54D4E90123C0
:10334000934280F048812268581C7821A060D154B3
:10335000D4E90123934280F039810F2F03D93A46F3
:1033600012090F2AFCD84FF0805603E036093FF4CB
:103370004BAEA3682168B7FBF6F2581CA0601BF89F
:103380000200C854D4E90131994206FB1277EDD30B
:103390002046FFF753FDE9E7DAF800301A1DCAF8B6
:1033A0000020D3F80080FB0740F197804746A7EB49
:1033B000080917F8013B002B75D0A2682168501C42
:1033C000A0608B54D4E901329A42F0D32046FFF733
:1033D00035FDECE7DAF80020111DCAF8001011687D
:1033E0002046CDE900670A22FFF76EFD0CE65A4938
:1033F0004FF49F70FEF75CFB6369002B7FF4F7AD21
:1034000055494FF4A070FEF753FB2368002B7FF45F
:10341000F2AD514940F24110FEF74AFBEBE5084698
:103420000026294630E6B8F1000F01DB780700D509
:10343000013E02B1D3B1F90718D4002E3FF470AFAA
:10344000B14513D220220393A1682368481CA060D1
:103450005A54D4E90131994206F1FF365DD2002E6B
:1034600000F0C480B145EFD1039B4E46B8F1000F88
:10347000C0F299807A070AD5A1684A1CA260226826
:103480002B205054D4E90121914280F0998007F01B
:103490000302022A66D0CDE9006741460A2220468F
:1034A000FFF712FDB0E54E457FF6AEAD202705E0F3
:1034B0004E453FF4A9AD002E3FF4A6ADA3682268A7
:1034C000591CA160D754D4E901329A4206F1FF3663
:1034D000EED32046FFF7B2FCEAE7B8F1000F24D0A4
:1034E000404602F05CF90746BE4220D9FEB14FF0DB
:1034F000200902E0BE421AD0CEB1A3682268591C4E
:10350000A16002F80390D4E901329A4206F1FF3635
:10351000F0D32046FFF792FCECE720460292FFF73B
:103520008DFC029A9BE70146B1E54746DCE708F1CE
:10353000FF3818F8013F002B3FF466ADA268216800
:10354000501CA0608B54D4E901329A42F1D320463A
:10355000FFF774FCEDE700BFB0670000CDCCCCCC2A
:10356000A0670000002B96D1002E3BD0B14592D22F
:1035700002932B464D469946A2682368501C4FF093
:103580003001A0609954D4E901329A4206F1FF3625
:1035900005D22EB3B542EFD1029B4D467BE72046C4
:1035A000FFF74CFCF5E7A1684A1CA26022682D20B9
:1035B0005054D4E901219142C8F10008FFF467AFEB
:1035C00020460293FFF73AFC029B60E72046FFF794
:1035D00035FCA368C1E62046FFF730FCA368B2E6DD
:1035E000029B4D46002656E71E463FE7039B97E6A3
:1035F0002DE9F041058BCE1C043D2E440746B6FB59
:10360000F5F6FEF701FB78B3F6B24FF48073013E96
:103610000446C5800760838027D08046002509E0E6
:103620006379AE4203F101036371C8F800000760DB
:1036300080461AD03846FEF7E7FA01350028EFD168
:103640006679721E14D02346013082421B68FBD17A
:103650001F684EB1002523682146013538461C46B7
:10366000FEF7FEFAAE42F6D100242046BDE8F08116
:103670002768EFE704300121FEF732BAF8B50121DF
:1036800004460430FEF738FAC0B200B1F8BD6679DE
:10369000721E12D02346013082421B68FBD11F6884
:1036A000002EF3D0002523682146013538461C46FC
:1036B000FEF7D6FAAE42F6D1F8BD2768F2E700BFB2
:1036C0002DE9F84F894692461D460446002843D00E
:1036D000B4F80680677908FB07F7043FBD4234D28F
:1036E0000AEB0503281D9F42B0FBF8F238BF7F1B91
:1036F00008FB120028BF574612B1013A2468FCD1DA
:10370000A8EB0005BD4228BF3D46A7B13E464FF09D
:10371000000B0430761B20442A4609EB0B0102F013
:1037200021F8B045AB44246845464FF0000028BF5F
:103730003546002EEDD1BA4505D00A49F620BDE840
:10374000F84FFEF7B5B9BDE8F88F0649C420FEF77B
:10375000AFF9B4F80680C3E70249B620FEF7A8F92E
:10376000B6E700BFE86700002DE9F84F89469246AA
:103770001D460446002844D0B4F80680677908FB4B
:1037800007F7043FBD4235D20AEB0503291D9F42CE
:10379000B1FBF8F238BF7F1B08FB121128BF574658
:1037A00012B1013A2468FCD1A8EB0105BD4228BF43
:1037B0003D46A7B13E464FF0000B04312144761B35
:1037C0002A4609EB0B0001F0CDFFB045AB4424685D
:1037D00045464FF0000128BF3546002EEDD1BA45D1
:1037E00006D00A494FF48070BDE8F84FFEF760B983
:1037F000BDE8F88F0549C420FEF75AF9B4F80680F1
:10380000C2E70249B620FEF753F9B5E7E8670000C2
:103810008368D3F83C319B076FD4012952D82DE936
:10382000F04F384B384D39495B1B9B08A1FB0323F4
:103830008DB0002B43D0C3EBC30305EB8303DFF84C
:10384000DCB00B9381462B68EA6809920020D3F81C
:103850000880AF68FEF7F8F82B681E685A68964231
:1038600049D9AB68013313449E1B0020FEF706F9CB
:10387000D5F814E095F810A0642404FB06FC5A4621
:1038800004FB08F47346B4FBF7F408214846BCFB7C
:10389000F7FC0A94BAF1000F18D11D4CCDF8148032
:1038A000CDE906740A9CCDE90374099C0094CDE926
:1038B00001C6FEF78DFD0B9B1C359D42C3D10DB09B
:1038C000BDE8F08F134A0221FEF782BD124BCDF8FE
:1038D0001480CDE906730A9BCDE90373099B00931D
:1038E000CDE901C673460821FEF772FD0B9B1C351E
:1038F0009D42A8D1E3E7961BB7E700221146FFF7E8
:10390000E1B800BF3C6C00003C6C000025499224EB
:10391000206900001C6000002C690000A468000001
:1039200010B5044610B12368986810BD03494FF4E0
:103930000670FEF7BDF82368986810BD686800003F
:1039400010B5044618B1236800229A6010BD0449DE
:1039500040F21E20FEF7ACF8236800229A6010BDEA
:103960006868000030B585B00478094A094B45689D
:103970008DF80040047AC068039053F82130019517
:103980008DF8084052F821106846984705B030BDC0
:10399000F4080020F808002030B585B004784568A8
:1039A0008DF80040D0E90240064A074B039053F8D7
:1039B000213001958DF8084052F82110684698474B
:1039C00005B030BDF4080020F8080020F0B51A4B0F
:1039D00006781A4D0C6991F81DE045F82640074617
:1039E000174803F806E040F826200C4694460FCC12
:1039F00089B06D460FC594E80F0085E80F00049666
:103A0000BEF1000F0BD0BCF1000F0E4A694607F162
:103A1000040008BF002201F0EDF909B0F0BDBCF1CF
:103A2000000F094A694607F10C0008BF002200F0A8
:103A3000F5FE09B0F0BD00BFC4090020F408002065
:103A4000F8080020653900009939000010B5154BC1
:103A50001A6882B07AB10021134A19601B68507944
:103A600000934FF080410123009CC1F8083310B946
:103A70001168537188470D4B1A6882B100221A6091
:103A80001B6801934FF080420221074B0198C2F856
:103A900008131B68012002B0BDE81040184702B0AF
:103AA00010BD00BF00010040FC08002004010040E0
:103AB0002DE9F04F89B00023AC4A03931168012926
:103AC00000F06C811E46AA4B1A68012A00F076812C
:103AD000A84B1A68012A00F08381A74B1A68012AB3
:103AE00000F09081A54B1A68012A00F09D81A44B3B
:103AF0001A68012A00F0AA81A24B1A68012A00F074
:103B0000B781A14B1A68012A0CD0A04B1B68012B6E
:103B100000F0BC8116F0FF0F15D1002E30DB09B08C
:103B2000BDE8F08F9A4AD2F804231706EDD500229B
:103B30001A601A6806926033069A1B68012B46F0D9
:103B4000800600F0A381934F00240125A30003F118
:103B50008043354203F5C0434FEA45050BD0D3F807
:103B6000100557F82420D3F81015C0F30420C1F332
:103B7000014102B190470134082CE7D1002ECEDA82
:103B800000224FF0FF33CDE90423824C824F4FF0E7
:103B9000010894F950305D1C32D0DBB223F0C00A2A
:103BA0004FEADA0208A901EB020B03F007091BF840
:103BB0000C5C08FA09F915EA090522D004EB0A01A0
:103BC0009E0991F9303054F82330002B00F09C818D
:103BD000032E00F09C81BAF11F0F00F2C1814FEA61
:103BE0008A0505F1A0451BF8142CD5F8001712EA38
:103BF0000909C1F3014140F05781032900F03682E1
:103C0000002594F95130581C32D0DBB223F0C00AA1
:103C100008A94FEADA0201EB020B03F007091BF8CF
:103C20000C1C08FA09F911EA090F21D004EB0A016A
:103C30009E0991F9303054F82330002B00F06D814B
:103C4000032E00F06D81BAF11F0F00F281814FEA5F
:103C50008A0202F1A0421BF8140CD2F8001710EAF5
:103C6000090FC1F3014140F02D81032900F0F881D3
:103C700094F95230591C32D0DBB223F0C00A08A9A3
:103C80004FEADA0201EB020B03F007091BF80C1CE8
:103C900008FA09F911EA090F21D004EB0A019E097B
:103CA00091F9303054F82330002B00F04881032E76
:103CB00000F04881BAF11F0F00F25A814FEA8A02E0
:103CC00002F1A0421BF8140CD2F8001710EA090FF9
:103CD000C1F3014140F00381032900F0BB8194F955
:103CE00053305A1C32D0DBB223F0C00A08A94FEA85
:103CF000DA0201EB020B03F007091BF80C1C08FAAF
:103D000009F911EA090F21D004EB0A019E0991F982
:103D1000303054F82330002B00F00881032E00F0DF
:103D20000881BAF11F0F00F22B814FEA8A0202F1DB
:103D3000A0421BF8140CD2F8001710EA090FC1F3C7
:103D4000014140F0D880032900F02281002D3FF48A
:103D5000E6AE4FF0A043039AD3F8103593423FF4F8
:103D6000DEAE049A0393059213E700BF00610040A2
:103D700004610040086100400C6100401061004097
:103D800014610040186100401C6100407C610040EB
:103D9000006000400409002074690000C249D1F8A5
:103DA000046316F001063FF48EAE136013680693A9
:103DB000069BBE4B1A68012A7FF48AAEBA4AD2F833
:103DC000042397077FF584AE00221A601B680693D0
:103DD000069BB74B1A68012A46F002067FF47DAEB7
:103DE000B14AD2F8042355077FF577AE00221A6056
:103DF0001B680693069BAF4B1A68012A46F004061F
:103E00007FF470AEA84AD2F8042314077FF56AAE97
:103E100000221A601B680693069BA74B1A68012AAA
:103E200046F008067FF463AE9F4AD2F80423D0061A
:103E30007FF55DAE00221A601B680693069B9F4BC0
:103E40001A68012A46F010067FF456AE964AD2F858
:103E5000042391067FF550AE00221A601B6806937A
:103E6000069B974B1A68012A46F020067FF449AE5C
:103E70008D4AD2F8042352067FF543AE00221A6021
:103E80001B680693069B46F040063AE68D4B0022DF
:103E90001A601B6807934FF0A043079AD3F81035B8
:103EA000039346F0004635E602297FF4A9AE032EBF
:103EB00000F00A810025002B3FF4A3AE31465046A6
:103EC00098479EE602297FF4D3AE032E00F0A2802D
:103ED000002B3FF4CDAE314650469847C8E6022944
:103EE0007FF4FDAE032E78D0002B3FF4F8AE3146C0
:103EF00050469847F3E602297FF428AF032E00F0DE
:103F0000A680002B65D121E7032E7FF479AE04A8AB
:103F1000815C41EA090181545DE6032E7FF4A8AE7D
:103F200004A8815C41EA090181548CE6032E7FF4E8
:103F30000DAF04A8815C41EA09018154F1E6032E2A
:103F40007FF4CDAE04A8815C41EA09018154B1E659
:103F500039464FF4E8700093FDF7AAFD009B76E622
:103F600039464FF4E8700093FDF7A2FD009B36E65A
:103F700039464FF4E8700093FDF79AFD009B9DE6EB
:103F800039464FF4E8700093FDF792FD009BCCE6B4
:103F9000032EB6D14FF40039BAF11F0F08D93946B4
:103FA0004FF4E870CDE90032FDF782FDDDE9003223
:103FB000D2F8001721F44031C2F80017D2F80017E8
:103FC000013541EA0901EDB2C2F80017002B3FF4B8
:103FD000C0AE314650469847B8E64FF44039BAF182
:103FE0001F0F08D939464FF4E870CDE90032FDF7CC
:103FF0005FFDDDE90032D2F8001721F44031C2F84C
:104000000017D2F80017013549EA0101EDB2C2F8F4
:10401000001769E74FF44039BAF11F0F08D9394644
:104020004FF4E870CDE90032FDF742FDDDE90032E2
:10403000D2F8001721F44031C2F80017D2F8001767
:10404000013549EA0101EDB2C2F8001740E74FF42B
:104050004039A1E7032E7FF447AF4FF40039BEE7A4
:10406000032E7FF435AF4FF40039D5E7032E7FF4EC
:1040700021AF4FF40039BAF11F0F06D939464FF47A
:10408000E8700093FDF714FD009BD5F8002722F49B
:104090004032C5F80027D5F8002749EA0202C5F8E2
:1040A0000027012507E700BF0060004004610040D1
:1040B000086100400C610040106100401461004044
:1040C000186100407C6100404FF44039D3E700BFE5
:1040D00010B5074C236813B1BDE8104018470549D7
:1040E0005120FDF7E5FC2368BDE81040184700BFEC
:1040F00060090020AC69000010B5044682B090B1A0
:10410000104B984202D0002002B010BD0020019157
:10411000FDF79AFC0C4B01991C795CB10020FDF76E
:10412000ADFC1120F0E709497720FDF7C1FC2046DE
:1041300002B010BD0122204619601A71FDF79EFCE5
:104140002046E1E70020004060090020AC69000043
:1041500040B1064B984200D07047054B00221A60D0
:104160001A71704703499B20FDF7A2BC0020004054
:1041700060090020AC6900002DE9F04701238B7233
:1041800091F809A0D0F80431002B8AB00E460546FC
:104190005FFA8AFA14BF0124002406D00023C0F875
:1041A0000431D0F804310093009BD5F82431002B62
:1041B0004FEA440414BF0123002306D00022C5F8AF
:1041C0002421D5F824210192019AD5F84C21002A06
:1041D00044EA432414BF0123002306D00022C5F87B
:1041E0004C21D5F84C210292029AD5F85021002A90
:1041F00044EAC34414BF0123002306D00022C5F8BB
:104200005021D5F850210392039AD5F86421002A51
:1042100044EA035414BF0123002306D00022C5F84A
:104220006421D5F864210492049AD5F86821002A03
:1042300044EA436414BF0123002306D00022C5F8DA
:104240006821D5F868210592059A54EA83643AD02A
:104250005A4FDFF86C91DFF86C810AF1FF3ABAF13E
:10426000030F19D8DFE80AF0363C020814EA090FF8
:104270007DD034F400245DD03C4278D0D5F83C3574
:104280003268DBB2042107938DF818100AB106A832
:10429000904734F0020432D014F00203F9D16001E7
:1042A00030D5E20232688DF8183056BF01234FF046
:1042B000020A9A468DF81C300AB106A8904724F0ED
:1042C000C364002CC9D1002386F809A0B3720AB0D8
:1042D000BDE8F08714EA080F32D034F480142CD0F3
:1042E0003C422DD0D5F84C353268DBB20121079322
:1042F0008DF81810002ACAD134F00204CCD14FF046
:10430000000AE0E7A30145D504F40023002B33683D
:104310004FF003020CBF012100218DF81C100CBFCF
:1043200092464FF0040A8DF81820002BC7D006A83B
:104330009847C4E74FF0040AC5E74FF0020AC2E706
:10434000D5F8D034C5F8D03472683168002B08BF76
:104350004FF480731A430220099372608DF8200095
:104360000029CCD008A888474FF0000AABE7D5F861
:10437000D034C5F8D03472683168002B08BF4FF4D0
:1043800080731A430520099372608DF8200000297C
:10439000E8D1B4E7D5F8D034C5F8D03472683168C4
:1043A000002B08BF4FF480731A43062009937260F4
:1043B0008DF820000029D5D1A1E700BF020000063A
:1043C000020008060200100603498B7A03B1704709
:1043D0000248FFF7D1BE00BF68090020003000404E
:1043E0002DE9F04F87B0054601920C46002900F0F8
:1043F000AA80D4E902239A4200F0918095F80480C3
:10440000DFF8B8A14FEA480606EB08030AEB83037E
:104410001B7A002B7DD12D6863492846FFF76CFE7F
:104420008146002840F089802B0B5AB25709BF0003
:10443000DBB207F1604702920393012207F561475F
:1044400003F01F0302FA03F34FF0FF32C5F8000533
:10445000C5F80825C5F80C25C7F88030C5F808232D
:10446000D4F808B0227CBBF11F0F7CD80BF5E07BA1
:1044700040F202614FF0A04041EA820240F82B2056
:10448000D4F80CB0627CBBF11F0F62D840F202611D
:104490004FF0A0400BF5E07B41EA820240F82B2070
:1044A000D4E9002152EA01003FD1012294F812B070
:1044B000BBF1070F61D802994FEA4B1B00295FFA45
:1044C0008BFB69DB01F1604101F5614181F800B3CB
:1044D000C7F880313B60D4E902134644C5F808159B
:1044E000C5F80C352378C5F88835B6000AEB060305
:1044F0002179019CC5F88C150120002118724846CD
:10450000C5F894254AF806409972597207B0BDE87B
:10451000F08F4FF00809484607B0BDE8F08F2349F7
:104520004FF4E970FDF7C4FA68E7003218BF0122C2
:104530000029BBD042F00202B8E74FF0110948460B
:1045400007B0BDE8F08F194940F2D110FDF7B0FA7D
:104550004FE717494FF4E870CDE90423FDF7A8FAB7
:10456000DDE9042392E712494FF4E870CDE9042312
:10457000FDF79EFADDE9042378E70E496B20CDE9CB
:104580000432FDF795FA02994FEA4B1B0029DDE949
:1045900004325FFA8BFB95DA0399074801F00F01AB
:1045A000084480F818B093E7C9430000EC690000A4
:1045B00074690000246A0000FCEC00E06809002037
:1045C000F0B50779234D04687E00F31905EB8303EA
:1045D00087B01B7A012B04D01F494FF41370FDF7ED
:1045E00067FA0023C4F80431D4F804210092009A39
:1045F000C4F82431D4F824210192019AC4F84C3132
:10460000D4F84C210292029AC4F85031D4F85021C7
:104610000392039AC4F86431D4F864210492F21925
:104620000499C4F86831D4F8681155F8223005911E
:10463000059A13B1094BC4F804333E4405EB8605D3
:10464000002302210922C4F8002529726B606B72D5
:1046500007B0F0BD68090020EC69000002021806EE
:1046600030B56C4AD2F8043399058BB066D5D2F8D0
:104670002431002B62D00023C2F82431D2F8243137
:1046800003934FF40171644B0398C2F8081393F835
:10469000291009B9012151605E4902228DF81820C4
:1046A000D1F88024C1F880249869D9680992002241
:1046B000CDE90710C3E90622D3E9001406A8A047F4
:1046C000544AD2F81C31BBB1534B186A596988421D
:1046D00069D350480022C0F81C21D0F81C01019079
:1046E000019849B198688DF8182008915A6107908F
:1046F000D3E9001206A89047464AD2F84431DBB10C
:104700000021454BC2F84411D2F8440193F8291016
:104710000090009809B1012111609A6962B10022EC
:10472000586AD9689A610122CDE907108DF81820DE
:1047300006A8D3E9001290470BB030BD354AD2F835
:1047400004335B07BCD5D2F80831002BB8D0324B0C
:10475000996900293CD00021C2F80811D2F808114B
:1047600004910499D868596AD2F8182542545A6AB3
:10477000996901325A625A6A8A42A1D1DA69196882
:10478000002A2ED0D8685D6A1C699A6107900022C1
:104790000120DC60DA615A628DF8180008955B68C8
:1047A00006A898478CE793F8280000F0FF0400283B
:1047B0008FD1C2F81C41D2F81C11029102999C6859
:1047C000186A196A205C01311962C2F81C0593E766
:1047D000C2F80811D2F8080105900598D2F81825FA
:1047E000C9E793F8292012B90A4A01205060094A02
:1047F0004FF40170C2F80803586ADA680890002480
:10480000012007928DF818005A689C6106A890470D
:1048100056E700BF00200040740900202DE9F04752
:10482000054684B091460C46002900F0E9802E79B7
:104830008E4F2C2303FB067393F82A30002B40F095
:10484000AA808B492868FFF757FC8046002840F073
:104850009C80D4F800A0BAF1FF3F17D0BAF11F0F27
:1048600000F2DF8001234FF0A04203FA0AF3C2F8FE
:104870000835D4F800A0BAF11F0F00F2CC800AF579
:10488000E07A4FF0A043032243F82A20D4F804A092
:10489000BAF1FF3F0AD0BAF11F0F00F2B6800AF555
:1048A000E07A4FF0A043002243F82A202B68A26947
:1048B000C3F82425217D637D2A680B43C2F86C353B
:1048C000D4E900122B68C3F81425C3F80C15237D16
:1048D000012B66D02C2303FB06F3FA18C2F80490D0
:1048E0002269FA50B9F1000F3BD02B68247F61494F
:1048F0000022C3F81C21D3F81C3102932B680298C4
:10490000C3F84421D3F844212B680392039AC3F8D7
:1049100004132B68072C4FEA133A4FFA8AF900F276
:104920009A806401B9F1000FE4B2C0F2998009F1F4
:10493000604303F5614383F800432A68120B42F396
:10494000C40323F0604323F0030303F1604303F542
:10495000614302F01F02012101FA02F2C3F8802133
:104960001A6029682C2303FB067604200023012209
:10497000C1F80005404686F82A20C6E9063386F8C5
:104980002930736104B0BDE8F0874FF0110840464C
:1049900004B0BDE8F0874FF00808404604B0BDE819
:1049A000F087D4F808A0BAF1FF3F09D0BAF11F0F81
:1049B0004BD80AF5E07A4FF0A043002243F82A20B2
:1049C000E3685A1C15D01F2B37D801224FF0A041A5
:1049D00002FA03F3C1F80835D4F80CA0BAF11F0F9E
:1049E00025D84FF0A0430AF5E07A032243F82A20A5
:1049F000E3682A68A168C2F80835C2F8101569E7AB
:104A00001D49AA20FDF754F811E71C494FF4E8703E
:104A1000FDF74EF843E719494FF4E870FDF748F801
:104A20002DE716494FF4E870FDF742F81AE71349ED
:104A30004FF4E870FDF73CF8D3E7104901934FF4C9
:104A4000E870FDF735F8019BBFE70C494FF4E870BB
:104A5000FDF72EF8ADE70A496B20FDF729F860E76E
:104A6000084B0AF00F0A53441C7666E774090020CD
:104A700061460000800002005C6A0000746900006A
:104A8000246A0000FCEC00E02DE9F047424E057975
:104A900002682C2303FB056300215B68C2F8001544
:104AA000044683B103683D4AC3F8082303683C48C1
:104AB0001B0B5AB25209203203F01F03012101FAE5
:104AC00003F340F8223023684FF0FF32D3F80CA5EF
:104AD000D3F81495D3F80875D3F81085C3F81425C6
:104AE000C3F80C2523689245C3F80825C3F81025A0
:104AF00009D0BAF11F0F49D80AF5E07A4FF0A04368
:104B0000022243F82A20B9F1FF3F09D0B9F11F0F63
:104B100036D809F5E0794FF0A043022243F8292066
:104B2000B8F1FF3F09D0B8F11F0F23D808F5E0789E
:104B30004FF0A043022243F828207B1C08D01F2FEF
:104B400012D807F5E0774FF0A043022243F8272060
:104B50002068FFF7FDFA2C2303FB0565002385F889
:104B60002A306B60BDE8F0870E494FF4E870FCF71F
:104B70009FFFE6E70B494FF4E870FCF799FFD5E794
:104B800008494FF4E870FCF793FFC2E705494FF47A
:104B9000E870FCF78DFFAFE7740900208402020083
:104BA00000E100E0746900002DE9F041454D06790F
:104BB0002C2303FB065384B093F82A30012B0446C0
:104BC0000F46904634D1002F74D0B8F1000F67D053
:104BD00021792C2303FB01514869002866D103FB8E
:104BE0000653012118629F6083F82800C3F81480DF
:104BF0002268C2F81C01D2F81C7122680297029F39
:104C000091602268D3F808C0C2F81C01D2F81C11C8
:104C100001910199D3F820E0196A5F681CF80EE051
:104C200001311962C2F81CE557B104B0BDE8F0814A
:104C3000254940F21510FCF73BFF002FC5D139E0A4
:104C40001A6A58692168904204D81AE093F828201B
:104C5000002A35D1D1F81C21002AF7D0C1F81C71E7
:104C6000D1F81C210392039AD3F820E01A6A1CF8A9
:104C70000EE001321A62C1F81CE51A6A8242E9D3D9
:104C80002168D1F81C31002BFBD00123CB60002020
:104C90002C2303FB065500236B6104B0BDE8F081B3
:104CA000094940F21710FCF703FF91E7112004B007
:104CB000BDE8F08104494FF48B70FCF7F9FE84E7FE
:104CC0000F20E5E7740900205C6A0000F0B5474B4F
:104CD000D3F8242189B0002A54D00021C3F824112C
:104CE000D3F82421029202228DF81020029AD3F8E0
:104CF00080043F4AC3F880040790D3F83C05D3688A
:104D00008DF81800C2E9061105931168536804A8CC
:104D10009847364BD3F84421BAB10020344AC3F83F
:104D20004401D3F8444191690194019C69B1D3F8DD
:104D30003C458DF81840D3689061012405931168B3
:104D400053688DF8104004A89847284BD3F82021C9
:104D5000B2B10021264AC3F82011D3F8204150698E
:104D60000094009C60B1D3F84C0593688DF818004E
:104D70008DF810105161059304A8D2E900139847EB
:104D800009B0F0BDD3F810110029C2D0C3F810212A
:104D9000D3F810111648039103998169D3F83C4563
:104DA0008C42B6D1C569C768D0E90016E4B295B1A6
:104DB000D3F800C285612CF02005C261C3F800520F
:104DC0000369C36001228DF8184005978DF8102003
:104DD00004A8B0479DE7012385618DF81840059729
:104DE0008DF8103004A8B04793E700BF00200040C2
:104DF000A00900202DE9F04F054687B092460C46E9
:104E0000002900F0F8802F79964E4FEAC70808EB8A
:104E1000070306EB830393F82030002B40F0B680A5
:104E200091492868FFF768F98146002840F0A8807A
:104E3000D4F800B0BBF1FF3F17D0BBF11F0F00F259
:104E4000EB8001234FF0A04203FA0BF3C2F80835C0
:104E5000D4F800B0BBF11F0F00F2D8800BF5E07B57
:104E60004FF0A043032243F82B20D4F804B0BBF149
:104E7000FF3F0AD0BBF11F0F00F2C2800BF5E07BB1
:104E80004FF0A043002243F82B202B68A269C3F8FF
:104E90002425217D637D2A680B43C2F86C35D4E953
:104EA00000212B68C3F80C25C3F81415237D012BB2
:104EB00072D008EB07039B00F218C2F804A0226925
:104EC000F250BAF1000F49D02A68247F67490023C5
:104ED000C2F81031D2F8102102922A680298C2F862
:104EE0002031D2F8202103922A680398C2F8243195
:104EF000D2F8242104922A680498C2F84431D2F8E6
:104F000044212B680592059AC3F804132B68072CDB
:104F10004FEA133B4FFA8BFA00F298806401BAF122
:104F2000000FE4B2C0F297800AF1604303F56143D9
:104F300083F800432A68120B42F3C40323F0604352
:104F400023F0030303F1604303F5614302F01F0202
:104F5000012101FA02F2C3F880211A60474406EBEE
:104F600087062A6801200023082186F82000484689
:104F7000C2F80015C6E90633736107B0BDE8F08FCB
:104F80004FF01109484607B0BDE8F08F4FF008090F
:104F9000484607B0BDE8F08FD4F808B0BBF1FF3F3A
:104FA00009D0BBF11F0F4BD80BF5E07B4FF0A043AE
:104FB000002243F82B20E268531C15D01F2A37D853
:104FC00001234FF0A04103FA02F2C1F80825D4F8FA
:104FD0000CB0BBF11F0F25D80BF5E07B4FF0A043C1
:104FE000032243F82B20E2682B68A168C3F8082548
:104FF000C3F810155DE71E49BC20FCF759FD02E718
:105000001C494FF4E870FCF753FD37E719494FF49A
:10501000E870FCF74DFD21E716494FF4E870FCF706
:1050200047FD0EE713494FF4E870FCF741FDD3E765
:10503000104901924FF4E870FCF73AFD019ABFE77E
:105040000C494FF4E870FCF733FDADE70A496B20DB
:10505000FCF72EFD62E7094B0BF00F0B5B441C764F
:1050600068E700BFA0090020CD4C0000100302003B
:105070009C6A000074690000246A0000FCEC00E0F7
:105080002DE9F84F90F80480434D02684FEAC806B6
:1050900006EB080305EB830300215B68C2F80015EB
:1050A000044683B103683D4AC3F8082303683C48BB
:1050B0001B0B5AB25209203203F01F03012101FADF
:1050C00003F340F8223023684FF0FF32D3F80CB5D9
:1050D000D3F814A5D3F80875D3F81095C3F80C25A8
:1050E000C3F8142523689345C3F80825C3F8102591
:1050F00009D0BBF11F0F49D80BF5E07B4FF0A0435F
:10510000022243F82B20BAF1FF3F09D0BAF11F0F5A
:1051100036D80AF5E07A4FF0A043022243F82A205D
:10512000B9F1FF3F09D0B9F11F0F23D809F5E07994
:105130004FF0A043022243F829207B1C08D01F2FE8
:1051400012D807F5E0774FF0A043022243F827205A
:10515000464405EB86052068FEF7FAFF002385F834
:1051600020306B60BDE8F88F0E494FF4E870FCF713
:105170009FFCE6E70B494FF4E870FCF799FCD5E794
:1051800008494FF4E870FCF793FCC2E705494FF477
:10519000E870FCF78DFCAFE7A009002010030200C7
:1051A00000E100E0746900002DE9F0430779424D09
:1051B000FE00F31905EB830383B093F82030012B35
:1051C00004468846914640D1B8F1000F53D0B9F15A
:1051D000000F47D0237913B9B9F1FF0F04D937492C
:1051E0004FF48870FCF764FC08F06043B3F1005F93
:1051F00034D1237903EBC30305EB830358690028FB
:105200003FD1F31905EB83030121C3F81490C3F8D0
:1052100008802268C2F82001D2F820210192226879
:10522000DDF804C0C2F85801D2F858210092226873
:10523000DDF800C0C2F84485C2F848952268916044
:105240005B6813B303B0BDE8F0831C4940F20D1056
:10525000FCF72EFCB8F1000FB9D10CE0102003B020
:10526000BDE8F083154940F20F10FCF721FC2379CB
:10527000002BB9D0B3E711494FF48770FCF718FC45
:10528000A5E7112003B0BDE8F083236800E08AB9E8
:10529000D3F82011D3F858210029F8D0002A14BFE0
:1052A0000F2000203E4405EB860500236B6103B010
:1052B000BDE8F0830F20F5E7A00900209C6A0000FC
:1052C000704700BF00B5084D0FCD87B001AC0FC4CB
:1052D0002B68064A0648236001A9FFF781F80448B5
:1052E000FFF76EF920BFFDE7DC6A0000C152000045
:1052F0001C00002030B4904B1B78062B20D08F4B25
:105300001B68062B00F085808D4AD2F8883043F464
:105310007003C2F88830BFF34F8FBFF36F8F4FF029
:105320001023D3F80022002AC0F28681D3F8043279
:10533000002BC0F28181834B834A1A6030BC7047D6
:10534000824B1B681D07DAD1814B1B6803F0F0020A
:10535000302A00F09E8003F0E003402B00F099809B
:105360007B4B1B6803F0F003302B00F0B980784BC7
:105370001B6803F0F002302A56D003F0E003402B04
:1053800052D0734B1B6803F0F003302B00F0B68053
:105390006F4B1B6803F0F002302A66D003F0E00385
:1053A000402B62D06A4B1B6803F0F003302B00F0F7
:1053B000B580674B1B6803F0F003302B79D0644B4A
:1053C0001B6803F0F003502B00F0E480604B1B6877
:1053D00003F0F002302A37D003F0E003402B33D043
:1053E0005B4B1B6803F0F002302A03D003F0E003AC
:1053F000402B84D14FF08043D3F80024D20744BF20
:105400006FF00102C3F800244C4B1B68062B7FF49D
:105410007BAF504B1B68062B7FF476AF4E4A136868
:1054200043F4806313606FE74C4B434A1B68127868
:105430004B49C3F34233062A0B6048D1434B1B68E8
:1054400019077FF45CAF9CE7464A3B4B12681B7818
:10545000454902F04F02062B0A607FF450AF3B4BE8
:105460001B6819077FF44BAFBAE74FF08043002267
:10547000C3F80C21C3F81021C3F838252E4B1B7834
:10548000062B7FF43CAF314B1B681B077FF437AF13
:1054900088E7364B284A1B6812783549C3F3042342
:1054A000062A0B60EAD1294B1B681C077FF427AF43
:1054B00056E7304C204A304912783048304B0525A9
:1054C000256001250D6000243F2104601960062A33
:1054D0007FF415AF1D4B1B681C077FF410AF6EE700
:1054E000154B284A1B7828491160062B7FF407AF1B
:1054F000164B1B6818077FF402AF38E723490E4BA1
:10550000CA681B7822F08072062BCA607FF4F7AE5F
:105510000E4B1B681A077FF4F2AE39E7064B1C4AA4
:105520001B780321062B11607FF4E9AE074B1B6843
:105530001D077FF4E4AE3CE7E00F00F030010010FF
:1055400000ED00E0240000200090D003E40F00F004
:10555000E80F00F0340100103C1700404402001036
:105560003C05004058020010E40E004024030010E7
:105570004035014010560040885600401856004003
:105580001456004074C007400DF0ADBAF0ED00E0D5
:10559000A00500404FF08053404AD3F80414C2F8ED
:1055A0002015D3F80814C2F82415D3F80C14C2F847
:1055B0002815D3F81014C2F82C15D3F81414C2F817
:1055C0003015D3F81814C2F83415D3F81C14C2F8E7
:1055D0004015D3F82014C2F84415D3F82414C2F8A7
:1055E0004815D3F82814C2F84C15D3F82C14C2F877
:1055F0005015D3F83014C2F85415D3F83414C2F847
:105600006015D3F83814C2F86415D3F83C14C2F806
:105610006815D3F840142248C2F86C15D3F8441426
:105620000378C2F87015062B7FF469AE1D4B1B681A
:1056300018077FF464AEC9E61B4B0122C3F80425AA
:10564000D3F80024002AFBD04FF01023152216496E
:10565000C3F80022D1F80034002BFBD04FF0102209
:105660001521114BC2F80412D3F80024002AFBD0F4
:1056700000220D49C3F80425D1F80034002BFBD0DB
:10568000BFF34F8F09490A4BCA6802F4E062134323
:10569000CB60BFF34F8F00BFFDE700BF00C00040ED
:1056A000E00F00F0E40F00F000E0014000ED00E04A
:1056B0000400FA0508B5074B044613B10021AFF307
:1056C0000080054B1868836A03B19847204600F0B4
:1056D0008DF800BF00000000F06A000070B50D4EAC
:1056E0000D4CA41BA4100025A54209D10B4E0C4C57
:1056F00000F07EF8A41BA4100025A54205D170BDC2
:1057000056F8253098470135EEE756F8253098478A
:105710000135F2E7F8010020F8010020F80100202F
:10572000FC010020044B054A1B681B6A002B08BFC4
:105730001346D3F8EC007047280000208C000020AE
:1057400082B001B901A942B14BB113780B60127854
:10575000101C18BF012002B070471046FBE76FF025
:105760000100F8E710B5431E0A44914200D110BD74
:1057700011F8014B03F8014FF7E702440346934247
:1057800000D1704703F8011BF9E710F8012B11F85D
:10579000013B012A28BF9A42F7D0D01A704703462E
:1057A00013F8012B002AFBD1181A0138704710B5E5
:1057B0006AB10139841810F8013B11F8012F9342A6
:1057C00003D1A04201D0002BF5D1981A10BD10468C
:1057D000FCE749B1FF2A85BF8A2303600A704FF0B6
:1057E000FF3098BF0120704708467047FEE700BFB2
:1057F000F8B500BFF8BC08BC9E467047F8B500BFBE
:10580000F8BC08BC9E467047FFFFFFFFFFFFFFFF8D
:10581000FFFFFFFFFFFFFFFF000000000000000090
:105820000000D60106010000C90300003504000095
:10583000C5030000756172745F6C6F675F626163BE
:105840006B656E6400000000656E61626C6500004F
:1058500042616420706172616D6574657220636F6E
:10586000756E742E0D0A000064697361626C6500C8
:10587000556E6B6E6F776E206F7074696F6E3A2025
:1058800025730D0A000000004C6576656C20756E6E
:10589000617661696C61626C6520666F72206D6F04
:1058A00064756C653A2025730D0A0000556E6B6EA9
:1058B0006F776E206D6F64756C653A25730D0A0005
:1058C000556E6B6E6F776E2073657665726974794D
:1058D000206C6576656C3A2025730D0A0000000087
:1058E000496E76616C6964206261636B656E643ACF
:1058F0002025730D0A00000025733A257325730DCA
:105900000A00000020756E6B6E6F776E20706172FA
:10591000616D657465723A2000000000656E616219
:105920006C65640064697361626C6564000000000A
:1059300025730D0A092D205374617475733A206420
:10594000656163746976617465640D0A0D0A00000F
:1059500025730D0A092D205374617475733A20253F
:10596000730D0A092D2049443A2025640D0A0D0AB9
:10597000000000004E6F7420737570706F72746554
:10598000642E0D0A000000002E2E2F2E2E2F2E2EFC
:105990002F2E2E2F2E2E2F2E2E2F636F6D706F6EAB
:1059A000656E74732F6C69627261726965732F6CB6
:1059B0006F672F7372632F6E72665F6C6F675F66BF
:1059C000726F6E74656E642E630000006E6F6E659C
:1059D000000000004C6F6773206172652068616C85
:1059E000746564210D0A00006D6F64756C655F6EEF
:1059F000616D6500252D343073207C2063757272D3
:105A0000656E74207C206275696C742D696E200D42
:105A10000A0000002D2D2D2D2D2D2D2D2D2D2D2D60
:105A20002D2D2D2D2D2D2D2D2D2D2D2D2D2D2D2DA6
:105A30002D2D2D2D2D2D2D2D2D2D2D2D2D2D2D2D96
:105A40002D2D2D2D2D2D2D2D2D2D2D2D2D2D0D0AC9
:105A500000000000252D343073207C20252D377365
:105A6000207C20257325730D0A0000002A00000009
:105A700001000000D104000001000000B107000097
:105A80000100000095040000CC590000545E0000A5
:105A9000645E00005C5E00004C5E00004C5E000036
:105AA000545E00005C5E0000CC590000645E0000A3
:105AB00000000000B85A000068580000785C000040
:105AC000785A0000A109000048580000E45C00007A
:105AD000805A0000A1090000685D00006C5D0000B4
:105AE000000000005D0700007C5D0000845D000098
:105AF000000000000D070000BC5D0000C45D000058
:105B00000000000045090000000000000000000047
:105B1000000000000000000000000000205B00000A
:105B2000D45D0000DC5D000000000000ED05000019
:105B3000105E0000185E0000000000000D0600006E
:105B40000000000000000000000000000000000055
:105B500000000000585B0000305C0000385C000072
:105B6000705A000000000000545C00005C5C000003
:105B7000185B00000000000068580000785C00001E
:105B8000785A00001D0C000048580000E45C00003A
:105B9000805A00001D0C0000685D00006C5D000074
:105BA00000000000C50400007C5D0000845D000072
:105BB00000000000B9040000945D0000A45D000036
:105BC0000000000059050000BC5D0000C45D00003D
:105BD0000000000039090000000000000000000083
:105BE00000000000000000000C5C0000105C0000E1
:105BF000505B0000190500004261636B656E6473C1
:105C000020666C7573686564000000006C6F670047
:105C1000436F6D6D616E647320666F7220636F6E8B
:105C200074726F6C6C696E67206C6F676765720069
:105C30006261636B656E64004C6F676765722062BA
:105C400061636B656E647320636F6D6D616E647309
:105C50002E000000636F6E66696700004D616E6123
:105C60006765206C6F6767657220636F6E66696732
:105C700075726174696F6E00276C6F672064697359
:105C800061626C65203C6D6F64756C655F303E20B1
:105C90002E2E203C6D6F64756C655F6E3E27206410
:105CA000697361626C6573206C6F677320696E2025
:105CB000737065636966696564206D6F64756C6592
:105CC000732028616C6C206966206E6F206D6F6494
:105CD000756C657320737065636966696564292EE8
:105CE00000000000276C6F6720656E61626C6520A4
:105CF0003C6C6576656C3E203C6D6F64756C655FD1
:105D0000303E202E2E2E20203C6D6F64756C655F1A
:105D10006E3E2720656E61626C6573206C6F6773E1
:105D200020757020746F20676976656E206C6576CB
:105D3000656C20696E2073706563696669656420AF
:105D40006D6F64756C65732028616C6C20696620CA
:105D50006E6F206D6F64756C657320737065636919
:105D600066696564292E0000676F000052657375CF
:105D70006D65206C6F6767696E67000068616C74A1
:105D80000000000048616C74206C6F6767696E6783
:105D9000000000006C6973745F6261636B656E6420
:105DA000730000004C69737473206C6F67676572D1
:105DB000206261636B656E64732E0000737461749E
:105DC000757300004C6F676765722073746174753A
:105DD000730000006C6F6164000000004C6F616430
:105DE00020636F6E66696775726174696F6E207388
:105DF000746F72656420696E206E6F6E2D766F6CA5
:105E00006174696C65206D656D6F72792E0000009C
:105E100073746F726500000053746F726520637550
:105E20007272656E7420636F6E66696775726174F5
:105E3000696F6E20696E206E6F6E2D766F6C617467
:105E4000696C65206D656D6F72792E006465627591
:105E5000670000006572726F72000000696E666F05
:105E6000000000007761726E696E670061707000FB
:105E70006C6F675F6D656D706F6F6C0062616C6CED
:105E80006F632E6C6F675F6D656D706F6F6C000078
:105E9000E85E0000105F0000C85E0000185F0000B0
:105EA000205F0000285F0000305F0000385F0000C6
:105EB000405F0000202530327800000020202000C4
:105EC0007C000000256300001B5B313B33316D001B
:105ED00025734C6F67732064726F7070656420283F
:105EE00025642925730D0A001B5B306D000000003E
:105EF0003C25733E2025733A20000000000000007E
:105F0000545E0000645E00005C5E00004C5E0000B9
:105F10001B5B313B33306D001B5B313B33326D001B
:105F20001B5B313B33336D001B5B313B33346D0006
:105F30001B5B313B33356D001B5B313B33366D00F2
:105F40001B5B313B33376D00466174616C206572B9
:105F5000726F720053797374656D20726573657426
:105F60000000000000000000000000000000000031
:105F70000338FDD8704700002E2E2F2E2E2F2E2EE8
:105F80002F2E2E2F2E2E2F2E2E2F636F6D706F6EB5
:105F9000656E74732F6C69627261726965732F75B7
:105FA00074696C2F6170705F7574696C5F706C617F
:105FB00074666F726D2E630000000000C05F000009
:105FC000BC5D0000F860000000000000411B000004
:105FD00000000000000000000000000000000000C1
:105FE0002E2E2F2E2E2F2E2E2F2E2E2F2E2E2F2ECC
:105FF0002E2F636F6D706F6E656E74732F6C696298
:106000007261726965732F62616C6C6F632F6E725F
:10601000665F62616C6C6F632E6300004261642096
:10602000617267756D656E7420636F756E740000C4
:1060300025730D0A092D20456C656D656E742073FE
:10604000697A653A092564202B20256420627974D9
:106050006573206F6620646562756720696E666F80
:10606000726D6174696F6E0D0A092D205573616739
:10607000653A092575252520282575206F7574201A
:106080006F6620257520656C656D656E7473290DCE
:106090000A092D204D6178696D756D3A09257525C0
:1060A0002520282575206F7574206F6620257520A2
:1060B000656C656D656E7473290D0A0D0A0000002C
:1060C000D0600000D8600000B85F0000411B0000F5
:1060D00062616C6C6F630000436F6D6D616E647321
:1060E00020666F722042414C4C4F43206D616E61BF
:1060F00067656D656E7400005072696E742073740C
:1061000061747573206F662062616C6C6F632069C7
:106110006E7374616E6365732E0000002E2E2F2E39
:106120002E2F2E2E2F2E2E2F2E2E2F2E2E2F636F14
:106130006D706F6E656E74732F6C696272617269D7
:1061400065732F636C692F6E72665F636C692E6373
:10615000000000001B4500001B5B6D001B5B48003E
:106160001B5B324A000000001B5B3F336C000000E9
:106170001B5B366E00000000202D20001B5B256499
:10618000420000001B5B2564440000001B5B25648B
:10619000430000001B5B256441000000000000007C
:1061A0000338FDD8704700002D682C202D2D686520
:1061B0006C70000000000000BC610000046600007C
:1061C0000C66000034620000D9290000246600003B
:1061D0002C6600006C6200009928000040660000F8
:1061E00048660000FC610000652A00000000000015
:1061F000000000000000000000000000000000009F
:1062000004620000586600006066000000000000A4
:10621000292700008C660000946600000000000042
:1062200061270000000000000000000000000000E6
:1062300000000000000000003C6200002C63000031
:1062400030670000000000003528000028630000CF
:1062500048670000000000006928000000000000FE
:10626000000000000000000000000000000000002E
:10627000746200002C630000C06600000000000093
:10628000F5260000286300001C67000000000000E5
:10629000C526000000000000000000000000000013
:1062A0000000000000000000AC620000B8650000C3
:1062B000C065000000000000D127000000000000C1
:1062C000000000000000000000000000A0650000C9
:1062D000A865000000000000392300007865000078
:1062E0007C650000B4610000212500004C6F7374D0
:1062F000206C6F67733A2025750D0A4D6178206C0C
:106300006F67207175657565207574696C697A6150
:1063100074696F6E3A2025752525205B25752F251C
:10632000755D0D0A000000006F6E00006F6666006C
:106330004563686F207374617475733A2025730D1B
:106340000A0000005B2533645D2025730D0A000000
:106350004E6F20726573706F6E73652066726F6D1D
:1063600020746865207465726D696E616C2C2061A3
:106370007373756D656420383078323420736372BE
:1063800065656E2073697A650D0A000025733A20F1
:1063900077726F6E6720706172616D6574657220CF
:1063A000636F756E740D0A004F7074696F6E733A87
:1063B0000D0A00002020252D2A733A0053686F77BC
:1063C00020636F6D6D616E642068656C702E0000D7
:1063D000537562636F6D6D616E64733A0D0A0000F0
:1063E0002020257325732573000000005C650000E4
:1063F0006465000000000000152900006E6F742025
:106400007465726D696E617465643A2025630D0A66
:1064100000000000257325730D0A00003A20636F09
:106420006D6D616E64206E6F7420666F756E6400B2
:106430002D6800002D2D68656C700000506C656142
:106440007365207370656369667920612073756276
:10645000636F6D6D616E642E0D0A000054616220E1
:1064600066756E6374696F6E3A20636F6D6D616EF1
:10647000647320636F756E746572206F76657266E3
:106480006C6F7765642E0D0A00000000202000006C
:106490000D0A2573257300000D0A25730000000006
:1064A000B4640000BC640000A46200008125000008
:1064B0002C200000726573697A650000436F6E736B
:1064C0006F6C652067657473207465726D696E61A9
:1064D0006C2073637265656E2073697A65206F72D4
:1064E00020617373756D657320383020696E206389
:1064F0006173652074686520726561646F757420CE
:106500006661696C732E204974206D757374206206
:10651000652065786563757465642061667465726D
:106520002065616368207465726D696E616C2077A7
:1065300069647468206368616E676520746F2065A4
:106540006E7375726520636F727265637420746513
:10655000787420646973706C61792E006869737453
:106560006F727900436F6D6D616E6420686973743A
:106570006F72792E00000000636C690055736566C8
:10658000756C2C206E6F7420556E69782D6C696B5C
:106590006520434C4920636F6D6D616E64732E00FE
:1065A000636C656172000000436C65617220736307
:1065B0007265656E2E00000064656661756C74001E
:1065C000417373756D652038302063686172732084
:1065D00073637265656E20776964746820616E64A8
:1065E0002073656E642074686973207365747469C0
:1065F0006E6720746F20746865207465726D696EB3
:10660000616C2E00636F6C6F72730000546F67676C
:106610006C6520636F6C6F7265642073796E746152
:10662000782E00006563686F00000000546F676794
:106630006C6520434C49206563686F2E00000000A4
:106640007374617473000000434C49207374617467
:106650006973746963732E0072657365740000005A
:10666000526573657420434C492073746174697377
:106670007469637320666F7220746865204C6F675D
:10668000676572206D6F64756C652E0073686F7737
:106690000000000047657420434C49207374617406
:1066A00069737469637320666F7220746865204C27
:1066B0006F67676572206D6F64756C652E000000F2
:1066C00044697361626C6520434C49206563686F5F
:1066D0002E204172726F777320616E642062757430
:1066E000746F6E733A204261636B73706163652CE3
:1066F0002044656C6574652C20456E642C20486FC1
:106700006D652C20496E7365727420617265206E10
:106710006F742068616E646C65642E00456E616202
:106720006C6520434C49206563686F2E00000000B3
:1067300044697361626C6520636F6C6F726564207D
:1067400073796E7461782E00456E61626C652063AA
:106750006F6C6F7265642073796E7461782E0000BF
:10676000636C695F75617274000000002E2E2F2E1D
:106770002E2F2E2E2F2E2E2F2E2E2F2E2E2F6578B3
:106780007465726E616C2F667072696E74662F6EBE
:1067900072665F667072696E74662E630000000038
:1067A0003031323334353637383941424344454647
:1067B0002E2E2F2E2E2F2E2E2F2E2E2F2E2E2F2EF4
:1067C0002E2F65787465726E616C2F667072696EBB
:1067D00074662F6E72665F667072696E74665F664D
:1067E0006F726D61742E63002E2E2F2E2E2F2E2E83
:1067F0002F2E2E2F2E2E2F2E2E2F636F6D706F6E3D
:10680000656E74732F6C69627261726965732F6D46
:10681000656D6F626A2F6E72665F6D656D6F626A1D
:106820002E6300007077725F6D676D74000000006A
:1068300038690000D860000040680000113800008E
:106840000000000048680000BC5D000040690000D6
:1068500000000000113800000000000000000000EF
:1068600000000000000000002E2E2F2E2E2F2E2EB6
:106870002F2E2E2F2E2E2F2E2E2F636F6D706F6EBC
:10688000656E74732F6C69627261726965732F71C2
:10689000756575652F6E72665F71756575652E63BA
:1068A0000000000025730D0A092D20456C656D65FB
:1068B0006E742073697A653A0925640D0A092D20E2
:1068C00055736167653A09257525252028257520AA
:1068D0006F7574206F6620257520656C656D656E1B
:1068E0007473290D0A092D204D6178696D756D3A13
:1068F000092575252520282575206F7574206F665C
:1069000020257520656C656D656E7473290D0A0907
:106910002D204D6F64653A090925730D0A0D0A0093
:106920004F766572666C6F77000000004E6F206FC7
:10693000766572666C6F770071756575650000002D
:106940005072696E7420737461747573206F662061
:10695000717565756520696E7374616E6365732EFC
:1069600000000000636C6F636B000000434C4F43FA
:106970004B0000002E2E2F2E2E2F2E2E2F2E2E2FA0
:106980002E2E2F2E2E2F6D6F64756C65732F6E72E9
:1069900066782F68616C2F6E72665F6770696F2E04
:1069A000680000004750494F544500002E2E2F2EFE
:1069B0002E2F2E2E2F2E2E2F2E2E2F2E2E2F6D6F72
:1069C00064756C65732F6E7266782F647269766574
:1069D00072732F7372632F7072732F6E7266785F8B
:1069E0007072732E63000000505253002E2E2F2E13
:1069F0002E2F2E2E2F2E2E2F2E2E2F2E2E2F6D6F32
:106A000064756C65732F6E7266782F647269766533
:106A100072732F7372632F6E7266785F7477697307
:106A20002E6300002E2E2F2E2E2F2E2E2F2E2E2FA9
:106A30002E2E2F2E2E2F696E746567726174696F0A
:106A40006E2F6E7266782F6E7266785F676C7565F2
:106A50002E68000054574953000000002E2E2F2EA0
:106A60002E2F2E2E2F2E2E2F2E2E2F2E2E2F6D6FC1
:106A700064756C65732F6E7266782F6472697665C3
:106A800072732F7372632F6E7266785F75617274A2
:106A90002E63000055415254000000002E2E2F2E70
:106AA0002E2F2E2E2F2E2E2F2E2E2F2E2E2F6D6F81
:106AB00064756C65732F6E7266782F647269766583
:106AC00072732F7372632F6E7266785F7561727462
:106AD000652E63005541525445000000030000003C
:106AE000000000000B0000000C0000000303060083
:106AF0002C0000204300504F534958002E00002026
:106B0000202020202020202028282828282020205D
:106B1000202020202020202020202020202020880D
:106B20001010101010101010101010101010100471
:106B300004040404040404040410101010101010C1
:106B400041414141414101010101010101010101B5
:106B500001010101010101010101101010101010CB
:106B60004242424242420202020202020202020285
:106B700002020202020202020202101010102000A1
:106B80000000000000000000000000000000000005
:106B900000000000000000000000000000000000F5
:106BA00000000000000000000000000000000000E5
:106BB00000000000000000000000000000000000D5
:106BC00000000000000000000000000000000000C5
:106BD00000000000000000000000000000000000B5
:106BE00000000000000000000000000000000000A5
:106BF0000000000000000000000000000000000095
:046C00000000000090
:106C040000000000E85B000000000000C06000001D
:106C140000000000A064000000000000EC6300001D
:106C240000000000DC62000000000000CC620000F4
:086C34000000000030680000C0
:106C3C006C69000000000000A46900000000000066
:106C4C00E869000000000000546A00000000000029
:106C5C00946A000000000000D46A000000000000EC
:106C6C006C5E0000000003037C5E0000000000036B
:106C7C006067000000000000646900000000000074
:086C8C00246800000000000074
:106C940028580000000000003458000014000020B0
:106CA400D8020020A0030020A8030020E002002056
:0C6CB40038020020705E00001800000094
:086CC0008095FF7F0100000038
:106CC80000000000002000400000000000200040FC
:106CD8000000000000000000FF000000003000403D
:106CE800000000000090D0032C00002000000000ED
:106CF800000000000000000000000000000000008C
:106D0800000000000000000000000000000000007B
:106D1800000000000000000000000000000000006B
:106D2800000000000000000000000000000000005B
:106D3800000000000000000000000000000000004B
:106D480000000000000000000000000043000000F8
:106D5800000000000000000000000000000000002B
:106D680000000000000000000000000043000000D8
:106D7800000000000000000000000000000000000B
:106D880000000000000000000000000043000000B8
:106D980000000000000000000000000000000000EB
:106DA8000000000000000000000000004300000098
:106DB80000000000000000000000000000000000CB
:106DC8000000000000000000000000004300000078
:106DD80000000000000000000000000000000000AB
:106DE8000000000000000000000000004300000058
:106DF800000000000000000000000000000000008B
:106E08000000000000000000000000004300000037
:106E1800000000000000000000000000000000006A
:106E2800000000000000000000000000D357000030
:106E38004157000000000000FE6A0000FC6A0000E4
:106E4800FD6A0000FD6A0000FD6A0000FD6A00009E
:106E5800FD6A0000FD6A0000FD6A0000FD6A00008E
:106E6800FD6A0000FFFFFFFFFFFFFFFFFFFFFFFFBF
:106E7800FFFF0000010041534349490000000000A2
:106E880000000000000000000000000000000000FA
:106E98000000000000004153434949000000000081
:106EA80000000000000000000000000000000000DA
:106EB80000000000000000002502000001020000A0
:106EC80000000000000000000000000000000000BA
:0C6ED800000000000000000000000000AE
:106EE400000000000000000000000000000000009E
:106EF400000000000000000000000000000000008E
:0C6F040000000000000000000000000081
:106F10000000000000000000000000000000000071
:106F20000000000000000000000000000000000061
:0C6F300000000000000000000000000055
:04000003000002B542
:00000001FF
